
C:\Documents and Settings\jarek\Pulpit\Privet\Magisterka\Programy\1\um0427\FWLib\project\RIDE\STM3210E-EVAL\MESSAGE.o:     file format elf32-littlearm
C:\Documents and Settings\jarek\Pulpit\Privet\Magisterka\Programy\1\um0427\FWLib\project\RIDE\STM3210E-EVAL\MESSAGE.o

Disassembly of section .text.InitTakNie:

00000000 <InitTakNie>:
InitTakNie():
C:\Documents and Settings\jarek\Pulpit\Privet\Magisterka\Programy\1\um0427\FWLib\project/MESSAGE.c:91
   0:	4b01      	ldr	r3, [pc, #4]	(8 <InitTakNie+0x8>)
   2:	2203      	movs	r2, #3
   4:	701a      	strb	r2, [r3, #0]
C:\Documents and Settings\jarek\Pulpit\Privet\Magisterka\Programy\1\um0427\FWLib\project/MESSAGE.c:92
   6:	4770      	bx	lr
   8:	00000000 	.word	0x00000000
Disassembly of section .text.InitTime:

00000000 <InitTime>:
InitTime():
C:\Documents and Settings\jarek\Pulpit\Privet\Magisterka\Programy\1\um0427\FWLib\project/MESSAGE.c:94
   0:	4b01      	ldr	r3, [pc, #4]	(8 <InitTime+0x8>)
   2:	220b      	movs	r2, #11
   4:	701a      	strb	r2, [r3, #0]
C:\Documents and Settings\jarek\Pulpit\Privet\Magisterka\Programy\1\um0427\FWLib\project/MESSAGE.c:95
   6:	4770      	bx	lr
   8:	00000000 	.word	0x00000000
Disassembly of section .text.InitOK:

00000000 <InitOK>:
InitOK():
C:\Documents and Settings\jarek\Pulpit\Privet\Magisterka\Programy\1\um0427\FWLib\project/MESSAGE.c:97
   0:	4b01      	ldr	r3, [pc, #4]	(8 <InitOK+0x8>)
   2:	2208      	movs	r2, #8
   4:	701a      	strb	r2, [r3, #0]
C:\Documents and Settings\jarek\Pulpit\Privet\Magisterka\Programy\1\um0427\FWLib\project/MESSAGE.c:98
   6:	4770      	bx	lr
   8:	00000000 	.word	0x00000000
Disassembly of section .text.InitEmpty:

00000000 <InitEmpty>:
InitEmpty():
C:\Documents and Settings\jarek\Pulpit\Privet\Magisterka\Programy\1\um0427\FWLib\project/MESSAGE.c:101
   0:	4b01      	ldr	r3, [pc, #4]	(8 <InitEmpty+0x8>)
   2:	2201      	movs	r2, #1
   4:	701a      	strb	r2, [r3, #0]
C:\Documents and Settings\jarek\Pulpit\Privet\Magisterka\Programy\1\um0427\FWLib\project/MESSAGE.c:102
   6:	4770      	bx	lr
   8:	00000000 	.word	0x00000000
Disassembly of section .text.InitString:

00000000 <InitString>:
InitString():
C:\Documents and Settings\jarek\Pulpit\Privet\Magisterka\Programy\1\um0427\FWLib\project/MESSAGE.c:105
   0:	4b01      	ldr	r3, [pc, #4]	(8 <InitString+0x8>)
   2:	2210      	movs	r2, #16
   4:	701a      	strb	r2, [r3, #0]
C:\Documents and Settings\jarek\Pulpit\Privet\Magisterka\Programy\1\um0427\FWLib\project/MESSAGE.c:106
   6:	4770      	bx	lr
   8:	00000000 	.word	0x00000000
Disassembly of section .text.DrawTime:

00000000 <DrawTime>:
DrawTime():
C:\Documents and Settings\jarek\Pulpit\Privet\Magisterka\Programy\1\um0427\FWLib\project/MESSAGE.c:913
   0:	e92d 4ff0 	stmdb	sp!, {r4, r5, r6, r7, r8, r9, sl, fp, lr}
   4:	4680      	mov	r8, r0
C:\Documents and Settings\jarek\Pulpit\Privet\Magisterka\Programy\1\um0427\FWLib\project/MESSAGE.c:916
   6:	2406      	movs	r4, #6
   8:	fb08 f404 	mul.w	r4, r8, r4
C:\Documents and Settings\jarek\Pulpit\Privet\Magisterka\Programy\1\um0427\FWLib\project/MESSAGE.c:913
   c:	460f      	mov	r7, r1
   e:	b085      	sub	sp, #20
C:\Documents and Settings\jarek\Pulpit\Privet\Magisterka\Programy\1\um0427\FWLib\project/MESSAGE.c:916
  10:	00fe      	lsls	r6, r7, #3
C:\Documents and Settings\jarek\Pulpit\Privet\Magisterka\Programy\1\um0427\FWLib\project/MESSAGE.c:913
  12:	4691      	mov	r9, r2
C:\Documents and Settings\jarek\Pulpit\Privet\Magisterka\Programy\1\um0427\FWLib\project/MESSAGE.c:916
  14:	2500      	movs	r5, #0
C:\Documents and Settings\jarek\Pulpit\Privet\Magisterka\Programy\1\um0427\FWLib\project/MESSAGE.c:913
  16:	469a      	mov	sl, r3
C:\Documents and Settings\jarek\Pulpit\Privet\Magisterka\Programy\1\um0427\FWLib\project/MESSAGE.c:915
  18:	f7ff fffe 	bl	0 <GRAPH_WhiteBlack>
C:\Documents and Settings\jarek\Pulpit\Privet\Magisterka\Programy\1\um0427\FWLib\project/MESSAGE.c:916
  1c:	4631      	mov	r1, r6
  1e:	220c      	movs	r2, #12
  20:	2308      	movs	r3, #8
  22:	4620      	mov	r0, r4
  24:	9500      	str	r5, [sp, #0]
  26:	f7ff fffe 	bl	0 <GRAPH_RectangleFilled>
C:\Documents and Settings\jarek\Pulpit\Privet\Magisterka\Programy\1\um0427\FWLib\project/MESSAGE.c:917
  2a:	4631      	mov	r1, r6
  2c:	220c      	movs	r2, #12
  2e:	2308      	movs	r3, #8
  30:	f104 0036 	add.w	r0, r4, #54	; 0x36
  34:	9500      	str	r5, [sp, #0]
  36:	f7ff fffe 	bl	0 <GRAPH_RectangleFilled>
C:\Documents and Settings\jarek\Pulpit\Privet\Magisterka\Programy\1\um0427\FWLib\project/MESSAGE.c:918
  3a:	220c      	movs	r2, #12
  3c:	2308      	movs	r3, #8
  3e:	4631      	mov	r1, r6
  40:	f104 0066 	add.w	r0, r4, #102	; 0x66
  44:	9500      	str	r5, [sp, #0]
  46:	f7ff fffe 	bl	0 <GRAPH_RectangleFilled>
C:\Documents and Settings\jarek\Pulpit\Privet\Magisterka\Programy\1\um0427\FWLib\project/MESSAGE.c:920
  4a:	4639      	mov	r1, r7
  4c:	4640      	mov	r0, r8
  4e:	f7ff fffe 	bl	0 <GRAPH_TextGoTo>
C:\Documents and Settings\jarek\Pulpit\Privet\Magisterka\Programy\1\um0427\FWLib\project/MESSAGE.c:921
  52:	f8d9 1000 	ldr.w	r1, [r9]
  56:	f44f 6461 	mov.w	r4, #3600	; 0xe10
  5a:	fbb1 f1f4 	udiv	r1, r1, r4
  5e:	f04f 0b18 	mov.w	fp, #24	; 0x18
  62:	fbb1 f3fb 	udiv	r3, r1, fp
  66:	fb03 111b 	mls	r1, r3, fp, r1
  6a:	483a      	ldr	r0, [pc, #232]	(ec <printf+0xec>)
  6c:	f7ff fffe 	bl	0 <printf>
C:\Documents and Settings\jarek\Pulpit\Privet\Magisterka\Programy\1\um0427\FWLib\project/MESSAGE.c:922
  70:	4839      	ldr	r0, [pc, #228]	(e8 <printf+0xe8>)
  72:	f7ff fffe 	bl	0 <printf>
C:\Documents and Settings\jarek\Pulpit\Privet\Magisterka\Programy\1\um0427\FWLib\project/MESSAGE.c:923
  76:	f108 0309 	add.w	r3, r8, #9	; 0x9
  7a:	4618      	mov	r0, r3
  7c:	4639      	mov	r1, r7
  7e:	9303      	str	r3, [sp, #12]
  80:	f7ff fffe 	bl	0 <GRAPH_TextGoTo>
C:\Documents and Settings\jarek\Pulpit\Privet\Magisterka\Programy\1\um0427\FWLib\project/MESSAGE.c:924
  84:	f8d9 3000 	ldr.w	r3, [r9]
  88:	353c      	adds	r5, #60
  8a:	fbb3 f1f4 	udiv	r1, r3, r4
  8e:	fb01 3114 	mls	r1, r1, r4, r3
  92:	4830      	ldr	r0, [pc, #192]	(154 <DrawTime+0x154>)
  94:	fbb1 f1f5 	udiv	r1, r1, r5
  98:	f7ff fffe 	bl	0 <printf>
C:\Documents and Settings\jarek\Pulpit\Privet\Magisterka\Programy\1\um0427\FWLib\project/MESSAGE.c:926
  9c:	f108 0611 	add.w	r6, r8, #17	; 0x11
C:\Documents and Settings\jarek\Pulpit\Privet\Magisterka\Programy\1\um0427\FWLib\project/MESSAGE.c:925
  a0:	482e      	ldr	r0, [pc, #184]	(bc <printf+0xbc>)
  a2:	f7ff fffe 	bl	0 <printf>
C:\Documents and Settings\jarek\Pulpit\Privet\Magisterka\Programy\1\um0427\FWLib\project/MESSAGE.c:926
  a6:	4639      	mov	r1, r7
  a8:	4630      	mov	r0, r6
  aa:	f7ff fffe 	bl	0 <GRAPH_TextGoTo>
C:\Documents and Settings\jarek\Pulpit\Privet\Magisterka\Programy\1\um0427\FWLib\project/MESSAGE.c:927
  ae:	f8d9 3000 	ldr.w	r3, [r9]
  b2:	4828      	ldr	r0, [pc, #160]	(154 <DrawTime+0x154>)
  b4:	fbb3 f1f4 	udiv	r1, r3, r4
  b8:	fb01 3114 	mls	r1, r1, r4, r3
  bc:	fbb1 f3f5 	udiv	r3, r1, r5
  c0:	fb03 1115 	mls	r1, r3, r5, r1
  c4:	f7ff fffe 	bl	0 <printf>
C:\Documents and Settings\jarek\Pulpit\Privet\Magisterka\Programy\1\um0427\FWLib\project/MESSAGE.c:928
  c8:	f7ff fffe 	bl	0 <GRAPH_WhiteBlack>
C:\Documents and Settings\jarek\Pulpit\Privet\Magisterka\Programy\1\um0427\FWLib\project/MESSAGE.c:929
  cc:	4824      	ldr	r0, [pc, #144]	(94 <printf+0x94>)
  ce:	f7ff fffe 	bl	0 <printf>
C:\Documents and Settings\jarek\Pulpit\Privet\Magisterka\Programy\1\um0427\FWLib\project/MESSAGE.c:931
  d2:	f1ba 0f02 	cmp.w	sl, #2	; 0x2
  d6:	d017      	beq.n	108 <DrawTime+0x108>
  d8:	f1ba 0f04 	cmp.w	sl, #4	; 0x4
  dc:	d024      	beq.n	128 <DrawTime+0x128>
  de:	f1ba 0f01 	cmp.w	sl, #1	; 0x1
  e2:	d132      	bne.n	14a <DrawTime+0x14a>
C:\Documents and Settings\jarek\Pulpit\Privet\Magisterka\Programy\1\um0427\FWLib\project/MESSAGE.c:935
  e4:	4639      	mov	r1, r7
  e6:	4630      	mov	r0, r6
  e8:	f7ff fffe 	bl	0 <GRAPH_TextGoTo>
C:\Documents and Settings\jarek\Pulpit\Privet\Magisterka\Programy\1\um0427\FWLib\project/MESSAGE.c:936
  ec:	f7ff fffe 	bl	0 <GRAPH_BlackWhite>
C:\Documents and Settings\jarek\Pulpit\Privet\Magisterka\Programy\1\um0427\FWLib\project/MESSAGE.c:937
  f0:	f8d9 3000 	ldr.w	r3, [r9]
  f4:	481b      	ldr	r0, [pc, #108]	(164 <DrawTime+0x164>)
  f6:	fbb3 f1f4 	udiv	r1, r3, r4
  fa:	fb01 3114 	mls	r1, r1, r4, r3
  fe:	fbb1 f3f5 	udiv	r3, r1, r5
 102:	fb03 1115 	mls	r1, r3, r5, r1
 106:	e01e      	b.n	146 <DrawTime+0x146>
C:\Documents and Settings\jarek\Pulpit\Privet\Magisterka\Programy\1\um0427\FWLib\project/MESSAGE.c:940
 108:	4639      	mov	r1, r7
 10a:	9803      	ldr	r0, [sp, #12]
 10c:	f7ff fffe 	bl	0 <GRAPH_TextGoTo>
C:\Documents and Settings\jarek\Pulpit\Privet\Magisterka\Programy\1\um0427\FWLib\project/MESSAGE.c:941
 110:	f7ff fffe 	bl	0 <GRAPH_BlackWhite>
C:\Documents and Settings\jarek\Pulpit\Privet\Magisterka\Programy\1\um0427\FWLib\project/MESSAGE.c:942
 114:	f8d9 3000 	ldr.w	r3, [r9]
 118:	4812      	ldr	r0, [pc, #72]	(164 <DrawTime+0x164>)
 11a:	fbb3 f1f4 	udiv	r1, r3, r4
 11e:	fb01 3114 	mls	r1, r1, r4, r3
 122:	fbb1 f1f5 	udiv	r1, r1, r5
 126:	e00e      	b.n	146 <DrawTime+0x146>
C:\Documents and Settings\jarek\Pulpit\Privet\Magisterka\Programy\1\um0427\FWLib\project/MESSAGE.c:945
 128:	4639      	mov	r1, r7
 12a:	4640      	mov	r0, r8
 12c:	f7ff fffe 	bl	0 <GRAPH_TextGoTo>
C:\Documents and Settings\jarek\Pulpit\Privet\Magisterka\Programy\1\um0427\FWLib\project/MESSAGE.c:946
 130:	f7ff fffe 	bl	0 <GRAPH_BlackWhite>
C:\Documents and Settings\jarek\Pulpit\Privet\Magisterka\Programy\1\um0427\FWLib\project/MESSAGE.c:947
 134:	f8d9 1000 	ldr.w	r1, [r9]
 138:	480a      	ldr	r0, [pc, #40]	(164 <DrawTime+0x164>)
 13a:	fbb1 f1f4 	udiv	r1, r1, r4
 13e:	fbb1 f3fb 	udiv	r3, r1, fp
 142:	fb03 111b 	mls	r1, r3, fp, r1
 146:	f7ff fffe 	bl	0 <printf>
C:\Documents and Settings\jarek\Pulpit\Privet\Magisterka\Programy\1\um0427\FWLib\project/MESSAGE.c:951
 14a:	f7ff fffe 	bl	0 <GRAPH_WhiteBlack>
C:\Documents and Settings\jarek\Pulpit\Privet\Magisterka\Programy\1\um0427\FWLib\project/MESSAGE.c:952
 14e:	b005      	add	sp, #20
 150:	e8bd 8ff0 	ldmia.w	sp!, {r4, r5, r6, r7, r8, r9, sl, fp, pc}
 154:	00000000 	.word	0x00000000
 158:	00000006 	.word	0x00000006
 15c:	0000000d 	.word	0x0000000d
 160:	00000013 	.word	0x00000013
 164:	00000018 	.word	0x00000018
Disassembly of section .text.DrawButton:

00000000 <DrawButton>:
DrawButton():
C:\Documents and Settings\jarek\Pulpit\Privet\Magisterka\Programy\1\um0427\FWLib\project/MESSAGE.c:877
   0:	e92d 4ff0 	stmdb	sp!, {r4, r5, r6, r7, r8, r9, sl, fp, lr}
   4:	2700      	movs	r7, #0
   6:	b089      	sub	sp, #36
   8:	9204      	str	r2, [sp, #16]
   a:	9006      	str	r0, [sp, #24]
   c:	9105      	str	r1, [sp, #20]
   e:	9303      	str	r3, [sp, #12]
  10:	463a      	mov	r2, r7
C:\Documents and Settings\jarek\Pulpit\Privet\Magisterka\Programy\1\um0427\FWLib\project/MESSAGE.c:881
  12:	9904      	ldr	r1, [sp, #16]
  14:	5653      	ldrsb	r3, [r2, r1]
  16:	b123      	cbz	r3, 22 <DrawButton+0x22>
C:\Documents and Settings\jarek\Pulpit\Privet\Magisterka\Programy\1\um0427\FWLib\project/MESSAGE.c:880
  18:	1c7b      	adds	r3, r7, #1
  1a:	b2df      	uxtb	r7, r3
  1c:	3201      	adds	r2, #1
  1e:	2fff      	cmp	r7, #255
  20:	d1f7      	bne.n	12 <DrawButton+0x12>
C:\Documents and Settings\jarek\Pulpit\Privet\Magisterka\Programy\1\um0427\FWLib\project/MESSAGE.c:886
  22:	9b03      	ldr	r3, [sp, #12]
  24:	b113      	cbz	r3, 2c <DrawButton+0x2c>
C:\Documents and Settings\jarek\Pulpit\Privet\Magisterka\Programy\1\um0427\FWLib\project/MESSAGE.c:887
  26:	f7ff fffe 	bl	0 <GRAPH_BlackWhite>
  2a:	e001      	b.n	6 <GRAPH_WhiteBlack+0x6>
C:\Documents and Settings\jarek\Pulpit\Privet\Magisterka\Programy\1\um0427\FWLib\project/MESSAGE.c:889
  2c:	f7ff fffe 	bl	0 <GRAPH_WhiteBlack>
C:\Documents and Settings\jarek\Pulpit\Privet\Magisterka\Programy\1\um0427\FWLib\project/MESSAGE.c:893
  30:	f04f 0806 	mov.w	r8, #6	; 0x6
  34:	9906      	ldr	r1, [sp, #24]
  36:	fb07 f408 	mul.w	r4, r7, r8
  3a:	fb01 fb08 	mul.w	fp, r1, r8
  3e:	9b05      	ldr	r3, [sp, #20]
  40:	1c61      	adds	r1, r4, #1
  42:	00de      	lsls	r6, r3, #3
  44:	f106 39ff 	add.w	r9, r6, #4294967295	; 0xffffffff
  48:	f10b 3aff 	add.w	sl, fp, #4294967295	; 0xffffffff
  4c:	9107      	str	r1, [sp, #28]
  4e:	2300      	movs	r3, #0
  50:	9300      	str	r3, [sp, #0]
  52:	4649      	mov	r1, r9
  54:	9a07      	ldr	r2, [sp, #28]
  56:	3309      	adds	r3, #9
  58:	4650      	mov	r0, sl
  5a:	f7ff fffe 	bl	0 <GRAPH_RectangleFilled>
C:\Documents and Settings\jarek\Pulpit\Privet\Magisterka\Programy\1\um0427\FWLib\project/MESSAGE.c:896
  5e:	2501      	movs	r5, #1
  60:	1eb1      	subs	r1, r6, #2
  62:	1ce2      	adds	r2, r4, #3
  64:	230b      	movs	r3, #11
  66:	f1ab 0002 	sub.w	r0, fp, #2	; 0x2
  6a:	9500      	str	r5, [sp, #0]
  6c:	f7ff fffe 	bl	0 <GRAPH_Rectangle>
C:\Documents and Settings\jarek\Pulpit\Privet\Magisterka\Programy\1\um0427\FWLib\project/MESSAGE.c:898
  70:	9b06      	ldr	r3, [sp, #24]
  72:	3609      	adds	r6, #9
  74:	18fc      	adds	r4, r7, r3
  76:	fb04 f408 	mul.w	r4, r4, r8
  7a:	1960      	adds	r0, r4, r5
  7c:	4649      	mov	r1, r9
  7e:	4633      	mov	r3, r6
  80:	4602      	mov	r2, r0
  82:	9500      	str	r5, [sp, #0]
  84:	f7ff fffe 	bl	0 <GRAPH_Line>
C:\Documents and Settings\jarek\Pulpit\Privet\Magisterka\Programy\1\um0427\FWLib\project/MESSAGE.c:900
  88:	4631      	mov	r1, r6
  8a:	4622      	mov	r2, r4
  8c:	4633      	mov	r3, r6
  8e:	4650      	mov	r0, sl
  90:	9500      	str	r5, [sp, #0]
  92:	f7ff fffe 	bl	0 <GRAPH_Line>
C:\Documents and Settings\jarek\Pulpit\Privet\Magisterka\Programy\1\um0427\FWLib\project/MESSAGE.c:903
  96:	9903      	ldr	r1, [sp, #12]
  98:	9a07      	ldr	r2, [sp, #28]
  9a:	2309      	movs	r3, #9
  9c:	9100      	str	r1, [sp, #0]
  9e:	4650      	mov	r0, sl
  a0:	4649      	mov	r1, r9
  a2:	f7ff fffe 	bl	0 <GRAPH_Rectangle>
C:\Documents and Settings\jarek\Pulpit\Privet\Magisterka\Programy\1\um0427\FWLib\project/MESSAGE.c:906
  a6:	9905      	ldr	r1, [sp, #20]
  a8:	9806      	ldr	r0, [sp, #24]
  aa:	f7ff fffe 	bl	0 <GRAPH_TextGoTo>
C:\Documents and Settings\jarek\Pulpit\Privet\Magisterka\Programy\1\um0427\FWLib\project/MESSAGE.c:907
  ae:	9804      	ldr	r0, [sp, #16]
  b0:	f7ff fffe 	bl	0 <printf>
C:\Documents and Settings\jarek\Pulpit\Privet\Magisterka\Programy\1\um0427\FWLib\project/MESSAGE.c:910
  b4:	f7ff fffe 	bl	0 <GRAPH_WhiteBlack>
C:\Documents and Settings\jarek\Pulpit\Privet\Magisterka\Programy\1\um0427\FWLib\project/MESSAGE.c:911
  b8:	b009      	add	sp, #36
  ba:	e8bd 8ff0 	ldmia.w	sp!, {r4, r5, r6, r7, r8, r9, sl, fp, pc}
  be:	46c0      	nop			(mov r8, r8)
Disassembly of section .text.DrawString:

00000000 <DrawString>:
DrawString():
C:\Documents and Settings\jarek\Pulpit\Privet\Magisterka\Programy\1\um0427\FWLib\project/MESSAGE.c:858
   0:	b570      	push	{r4, r5, r6, lr}
C:\Documents and Settings\jarek\Pulpit\Privet\Magisterka\Programy\1\um0427\FWLib\project/MESSAGE.c:859
   2:	4604      	mov	r4, r0
   4:	4d18      	ldr	r5, [pc, #96]	(68 <DrawString+0x68>)
   6:	b1e8      	cbz	r0, 44 <DrawString+0x44>
C:\Documents and Settings\jarek\Pulpit\Privet\Magisterka\Programy\1\um0427\FWLib\project/MESSAGE.c:860
   8:	f7ff fffe 	bl	0 <GRAPH_WhiteBlack>
C:\Documents and Settings\jarek\Pulpit\Privet\Magisterka\Programy\1\um0427\FWLib\project/MESSAGE.c:861
   c:	2107      	movs	r1, #7
   e:	2009      	movs	r0, #9
  10:	f7ff fffe 	bl	0 <GRAPH_TextGoTo>
C:\Documents and Settings\jarek\Pulpit\Privet\Magisterka\Programy\1\um0427\FWLib\project/MESSAGE.c:862
  14:	4815      	ldr	r0, [pc, #84]	(58 <printf+0x58>)
  16:	f7ff fffe 	bl	0 <printf>
C:\Documents and Settings\jarek\Pulpit\Privet\Magisterka\Programy\1\um0427\FWLib\project/MESSAGE.c:863
  1a:	2107      	movs	r1, #7
  1c:	2009      	movs	r0, #9
  1e:	f7ff fffe 	bl	0 <GRAPH_TextGoTo>
C:\Documents and Settings\jarek\Pulpit\Privet\Magisterka\Programy\1\um0427\FWLib\project/MESSAGE.c:864
  22:	6ae8      	ldr	r0, [r5, #44]
  24:	f7ff fffe 	bl	0 <printf>
C:\Documents and Settings\jarek\Pulpit\Privet\Magisterka\Programy\1\um0427\FWLib\project/MESSAGE.c:865
  28:	f7ff fffe 	bl	0 <GRAPH_BlackWhite>
C:\Documents and Settings\jarek\Pulpit\Privet\Magisterka\Programy\1\um0427\FWLib\project/MESSAGE.c:866
  2c:	f104 0008 	add.w	r0, r4, #8	; 0x8
  30:	2107      	movs	r1, #7
  32:	f7ff fffe 	bl	0 <GRAPH_TextGoTo>
C:\Documents and Settings\jarek\Pulpit\Privet\Magisterka\Programy\1\um0427\FWLib\project/MESSAGE.c:867
  36:	6aeb      	ldr	r3, [r5, #44]
  38:	18e3      	adds	r3, r4, r3
  3a:	f913 0c01 	ldrsb.w	r0, [r3, #-1]
  3e:	f7ff fffe 	bl	0 <GRAPH_WriteChar>
  42:	e00f      	b.n	22 <GRAPH_WhiteBlack+0x22>
C:\Documents and Settings\jarek\Pulpit\Privet\Magisterka\Programy\1\um0427\FWLib\project/MESSAGE.c:869
  44:	f7ff fffe 	bl	0 <GRAPH_WhiteBlack>
C:\Documents and Settings\jarek\Pulpit\Privet\Magisterka\Programy\1\um0427\FWLib\project/MESSAGE.c:870
  48:	2107      	movs	r1, #7
  4a:	2009      	movs	r0, #9
  4c:	f7ff fffe 	bl	0 <GRAPH_TextGoTo>
C:\Documents and Settings\jarek\Pulpit\Privet\Magisterka\Programy\1\um0427\FWLib\project/MESSAGE.c:871
  50:	4806      	ldr	r0, [pc, #24]	(1c <printf+0x1c>)
  52:	f7ff fffe 	bl	0 <printf>
C:\Documents and Settings\jarek\Pulpit\Privet\Magisterka\Programy\1\um0427\FWLib\project/MESSAGE.c:872
  56:	2009      	movs	r0, #9
  58:	2107      	movs	r1, #7
  5a:	f7ff fffe 	bl	0 <GRAPH_TextGoTo>
C:\Documents and Settings\jarek\Pulpit\Privet\Magisterka\Programy\1\um0427\FWLib\project/MESSAGE.c:873
  5e:	6ae8      	ldr	r0, [r5, #44]
  60:	f7ff fffe 	bl	0 <printf>
C:\Documents and Settings\jarek\Pulpit\Privet\Magisterka\Programy\1\um0427\FWLib\project/MESSAGE.c:875
  64:	bd70      	pop	{r4, r5, r6, pc}
  66:	46c0      	nop			(mov r8, r8)
  68:	00000000 	.word	0x00000000
  6c:	0000001d 	.word	0x0000001d
Disassembly of section .text.StringUP:

00000000 <StringUP>:
StringUP():
C:\Documents and Settings\jarek\Pulpit\Privet\Magisterka\Programy\1\um0427\FWLib\project/MESSAGE.c:836
   0:	4a20      	ldr	r2, [pc, #128]	(84 <StringUP+0x84>)
   2:	4b21      	ldr	r3, [pc, #132]	(88 <StringUP+0x88>)
   4:	2100      	movs	r1, #0
   6:	6059      	str	r1, [r3, #4]
C:\Documents and Settings\jarek\Pulpit\Privet\Magisterka\Programy\1\um0427\FWLib\project/MESSAGE.c:837
   8:	6ad3      	ldr	r3, [r2, #44]
C:\Documents and Settings\jarek\Pulpit\Privet\Magisterka\Programy\1\um0427\FWLib\project/MESSAGE.c:835
   a:	e92d 41f0 	stmdb	sp!, {r4, r5, r6, r7, r8, lr}
C:\Documents and Settings\jarek\Pulpit\Privet\Magisterka\Programy\1\um0427\FWLib\project/MESSAGE.c:837
   e:	3b01      	subs	r3, #1
C:\Documents and Settings\jarek\Pulpit\Privet\Magisterka\Programy\1\um0427\FWLib\project/MESSAGE.c:835
  10:	4605      	mov	r5, r0
C:\Documents and Settings\jarek\Pulpit\Privet\Magisterka\Programy\1\um0427\FWLib\project/MESSAGE.c:836
  12:	6d57      	ldr	r7, [r2, #84]
C:\Documents and Settings\jarek\Pulpit\Privet\Magisterka\Programy\1\um0427\FWLib\project/MESSAGE.c:837
  14:	181c      	adds	r4, r3, r0
  16:	f102 0658 	add.w	r6, r2, #88	; 0x58
C:\Documents and Settings\jarek\Pulpit\Privet\Magisterka\Programy\1\um0427\FWLib\project/MESSAGE.c:836
  1a:	e006      	b.n	2a <StringUP+0x2a>
C:\Documents and Settings\jarek\Pulpit\Privet\Magisterka\Programy\1\um0427\FWLib\project/MESSAGE.c:837
  1c:	f994 2000 	ldrsb.w	r2, [r4]
  20:	f916 3b01 	ldrsb.w	r3, [r6], #1
  24:	1c41      	adds	r1, r0, #1
  26:	429a      	cmp	r2, r3
  28:	d002      	beq.n	30 <StringUP+0x30>
C:\Documents and Settings\jarek\Pulpit\Privet\Magisterka\Programy\1\um0427\FWLib\project/MESSAGE.c:836
  2a:	42b9      	cmp	r1, r7
C:\Documents and Settings\jarek\Pulpit\Privet\Magisterka\Programy\1\um0427\FWLib\project/MESSAGE.c:837
  2c:	4608      	mov	r0, r1
C:\Documents and Settings\jarek\Pulpit\Privet\Magisterka\Programy\1\um0427\FWLib\project/MESSAGE.c:836
  2e:	dbf5      	blt.n	1c <StringUP+0x1c>
  30:	4b15      	ldr	r3, [pc, #84]	(88 <StringUP+0x88>)
C:\Documents and Settings\jarek\Pulpit\Privet\Magisterka\Programy\1\um0427\FWLib\project/MESSAGE.c:841
  32:	4915      	ldr	r1, [pc, #84]	(88 <StringUP+0x88>)
C:\Documents and Settings\jarek\Pulpit\Privet\Magisterka\Programy\1\um0427\FWLib\project/MESSAGE.c:836
  34:	6058      	str	r0, [r3, #4]
C:\Documents and Settings\jarek\Pulpit\Privet\Magisterka\Programy\1\um0427\FWLib\project/MESSAGE.c:841
  36:	1c43      	adds	r3, r0, #1
C:\Documents and Settings\jarek\Pulpit\Privet\Magisterka\Programy\1\um0427\FWLib\project/MESSAGE.c:842
  38:	429f      	cmp	r7, r3
C:\Documents and Settings\jarek\Pulpit\Privet\Magisterka\Programy\1\um0427\FWLib\project/MESSAGE.c:841
  3a:	604b      	str	r3, [r1, #4]
  3c:	4a11      	ldr	r2, [pc, #68]	(84 <StringUP+0x84>)
C:\Documents and Settings\jarek\Pulpit\Privet\Magisterka\Programy\1\um0427\FWLib\project/MESSAGE.c:842
  3e:	d104      	bne.n	4a <StringUP+0x4a>
C:\Documents and Settings\jarek\Pulpit\Privet\Magisterka\Programy\1\um0427\FWLib\project/MESSAGE.c:843
  40:	2300      	movs	r3, #0
  42:	604b      	str	r3, [r1, #4]
C:\Documents and Settings\jarek\Pulpit\Privet\Magisterka\Programy\1\um0427\FWLib\project/MESSAGE.c:844
  44:	f892 3058 	ldrb.w	r3, [r2, #88]
  48:	e002      	b.n	50 <StringUP+0x50>
C:\Documents and Settings\jarek\Pulpit\Privet\Magisterka\Programy\1\um0427\FWLib\project/MESSAGE.c:847
  4a:	189b      	adds	r3, r3, r2
  4c:	f893 3058 	ldrb.w	r3, [r3, #88]
  50:	7023      	strb	r3, [r4, #0]
C:\Documents and Settings\jarek\Pulpit\Privet\Magisterka\Programy\1\um0427\FWLib\project/MESSAGE.c:852
  52:	4c0c      	ldr	r4, [pc, #48]	(84 <StringUP+0x84>)
C:\Documents and Settings\jarek\Pulpit\Privet\Magisterka\Programy\1\um0427\FWLib\project/MESSAGE.c:850
  54:	f7ff fffe 	bl	0 <GRAPH_WhiteBlack>
C:\Documents and Settings\jarek\Pulpit\Privet\Magisterka\Programy\1\um0427\FWLib\project/MESSAGE.c:851
  58:	2107      	movs	r1, #7
  5a:	2009      	movs	r0, #9
  5c:	f7ff fffe 	bl	0 <GRAPH_TextGoTo>
C:\Documents and Settings\jarek\Pulpit\Privet\Magisterka\Programy\1\um0427\FWLib\project/MESSAGE.c:852
  60:	6ae0      	ldr	r0, [r4, #44]
  62:	f7ff fffe 	bl	0 <printf>
C:\Documents and Settings\jarek\Pulpit\Privet\Magisterka\Programy\1\um0427\FWLib\project/MESSAGE.c:853
  66:	f7ff fffe 	bl	0 <GRAPH_BlackWhite>
C:\Documents and Settings\jarek\Pulpit\Privet\Magisterka\Programy\1\um0427\FWLib\project/MESSAGE.c:854
  6a:	f105 0008 	add.w	r0, r5, #8	; 0x8
  6e:	2107      	movs	r1, #7
  70:	f7ff fffe 	bl	0 <GRAPH_TextGoTo>
C:\Documents and Settings\jarek\Pulpit\Privet\Magisterka\Programy\1\um0427\FWLib\project/MESSAGE.c:855
  74:	6ae3      	ldr	r3, [r4, #44]
  76:	18eb      	adds	r3, r5, r3
  78:	f913 0c01 	ldrsb.w	r0, [r3, #-1]
  7c:	f7ff fffe 	bl	0 <GRAPH_WriteChar>
C:\Documents and Settings\jarek\Pulpit\Privet\Magisterka\Programy\1\um0427\FWLib\project/MESSAGE.c:856
  80:	e8bd 81f0 	ldmia.w	sp!, {r4, r5, r6, r7, r8, pc}
	...
Disassembly of section .text.StringDOWN:

00000000 <StringDOWN>:
StringDOWN():
C:\Documents and Settings\jarek\Pulpit\Privet\Magisterka\Programy\1\um0427\FWLib\project/MESSAGE.c:811
   0:	4a22      	ldr	r2, [pc, #136]	(8c <StringDOWN+0x8c>)
   2:	4b23      	ldr	r3, [pc, #140]	(90 <StringDOWN+0x90>)
   4:	2100      	movs	r1, #0
   6:	6059      	str	r1, [r3, #4]
C:\Documents and Settings\jarek\Pulpit\Privet\Magisterka\Programy\1\um0427\FWLib\project/MESSAGE.c:812
   8:	6ad3      	ldr	r3, [r2, #44]
C:\Documents and Settings\jarek\Pulpit\Privet\Magisterka\Programy\1\um0427\FWLib\project/MESSAGE.c:810
   a:	e92d 41f0 	stmdb	sp!, {r4, r5, r6, r7, r8, lr}
C:\Documents and Settings\jarek\Pulpit\Privet\Magisterka\Programy\1\um0427\FWLib\project/MESSAGE.c:812
   e:	3b01      	subs	r3, #1
C:\Documents and Settings\jarek\Pulpit\Privet\Magisterka\Programy\1\um0427\FWLib\project/MESSAGE.c:810
  10:	4606      	mov	r6, r0
C:\Documents and Settings\jarek\Pulpit\Privet\Magisterka\Programy\1\um0427\FWLib\project/MESSAGE.c:811
  12:	6d54      	ldr	r4, [r2, #84]
C:\Documents and Settings\jarek\Pulpit\Privet\Magisterka\Programy\1\um0427\FWLib\project/MESSAGE.c:812
  14:	181d      	adds	r5, r3, r0
  16:	f102 0758 	add.w	r7, r2, #88	; 0x58
C:\Documents and Settings\jarek\Pulpit\Privet\Magisterka\Programy\1\um0427\FWLib\project/MESSAGE.c:811
  1a:	e006      	b.n	2a <StringDOWN+0x2a>
C:\Documents and Settings\jarek\Pulpit\Privet\Magisterka\Programy\1\um0427\FWLib\project/MESSAGE.c:812
  1c:	f995 2000 	ldrsb.w	r2, [r5]
  20:	f917 3b01 	ldrsb.w	r3, [r7], #1
  24:	1c41      	adds	r1, r0, #1
  26:	429a      	cmp	r2, r3
  28:	d002      	beq.n	30 <StringDOWN+0x30>
C:\Documents and Settings\jarek\Pulpit\Privet\Magisterka\Programy\1\um0427\FWLib\project/MESSAGE.c:811
  2a:	42a1      	cmp	r1, r4
C:\Documents and Settings\jarek\Pulpit\Privet\Magisterka\Programy\1\um0427\FWLib\project/MESSAGE.c:812
  2c:	4608      	mov	r0, r1
C:\Documents and Settings\jarek\Pulpit\Privet\Magisterka\Programy\1\um0427\FWLib\project/MESSAGE.c:811
  2e:	dbf5      	blt.n	1c <StringDOWN+0x1c>
  30:	4b17      	ldr	r3, [pc, #92]	(90 <StringDOWN+0x90>)
  32:	4a17      	ldr	r2, [pc, #92]	(90 <StringDOWN+0x90>)
  34:	6058      	str	r0, [r3, #4]
C:\Documents and Settings\jarek\Pulpit\Privet\Magisterka\Programy\1\um0427\FWLib\project/MESSAGE.c:817
  36:	1e43      	subs	r3, r0, #1
  38:	429c      	cmp	r4, r3
  3a:	d103      	bne.n	44 <StringDOWN+0x44>
C:\Documents and Settings\jarek\Pulpit\Privet\Magisterka\Programy\1\um0427\FWLib\project/MESSAGE.c:818
  3c:	2300      	movs	r3, #0
  3e:	6053      	str	r3, [r2, #4]
C:\Documents and Settings\jarek\Pulpit\Privet\Magisterka\Programy\1\um0427\FWLib\project/MESSAGE.c:819
  40:	4b12      	ldr	r3, [pc, #72]	(8c <StringDOWN+0x8c>)
  42:	e007      	b.n	54 <StringDOWN+0x54>
C:\Documents and Settings\jarek\Pulpit\Privet\Magisterka\Programy\1\um0427\FWLib\project/MESSAGE.c:822
  44:	2b00      	cmp	r3, #0
C:\Documents and Settings\jarek\Pulpit\Privet\Magisterka\Programy\1\um0427\FWLib\project/MESSAGE.c:821
  46:	6053      	str	r3, [r2, #4]
C:\Documents and Settings\jarek\Pulpit\Privet\Magisterka\Programy\1\um0427\FWLib\project/MESSAGE.c:822
  48:	da01      	bge.n	4e <StringDOWN+0x4e>
C:\Documents and Settings\jarek\Pulpit\Privet\Magisterka\Programy\1\um0427\FWLib\project/MESSAGE.c:823
  4a:	1e63      	subs	r3, r4, #1
  4c:	6053      	str	r3, [r2, #4]
C:\Documents and Settings\jarek\Pulpit\Privet\Magisterka\Programy\1\um0427\FWLib\project/MESSAGE.c:825
  4e:	6853      	ldr	r3, [r2, #4]
  50:	4a0e      	ldr	r2, [pc, #56]	(8c <StringDOWN+0x8c>)
  52:	189b      	adds	r3, r3, r2
  54:	f893 3058 	ldrb.w	r3, [r3, #88]
C:\Documents and Settings\jarek\Pulpit\Privet\Magisterka\Programy\1\um0427\FWLib\project/MESSAGE.c:830
  58:	4c0c      	ldr	r4, [pc, #48]	(8c <StringDOWN+0x8c>)
C:\Documents and Settings\jarek\Pulpit\Privet\Magisterka\Programy\1\um0427\FWLib\project/MESSAGE.c:825
  5a:	702b      	strb	r3, [r5, #0]
C:\Documents and Settings\jarek\Pulpit\Privet\Magisterka\Programy\1\um0427\FWLib\project/MESSAGE.c:828
  5c:	f7ff fffe 	bl	0 <GRAPH_WhiteBlack>
C:\Documents and Settings\jarek\Pulpit\Privet\Magisterka\Programy\1\um0427\FWLib\project/MESSAGE.c:829
  60:	2107      	movs	r1, #7
  62:	2009      	movs	r0, #9
  64:	f7ff fffe 	bl	0 <GRAPH_TextGoTo>
C:\Documents and Settings\jarek\Pulpit\Privet\Magisterka\Programy\1\um0427\FWLib\project/MESSAGE.c:830
  68:	6ae0      	ldr	r0, [r4, #44]
  6a:	f7ff fffe 	bl	0 <printf>
C:\Documents and Settings\jarek\Pulpit\Privet\Magisterka\Programy\1\um0427\FWLib\project/MESSAGE.c:831
  6e:	f7ff fffe 	bl	0 <GRAPH_BlackWhite>
C:\Documents and Settings\jarek\Pulpit\Privet\Magisterka\Programy\1\um0427\FWLib\project/MESSAGE.c:832
  72:	f106 0008 	add.w	r0, r6, #8	; 0x8
  76:	2107      	movs	r1, #7
  78:	f7ff fffe 	bl	0 <GRAPH_TextGoTo>
C:\Documents and Settings\jarek\Pulpit\Privet\Magisterka\Programy\1\um0427\FWLib\project/MESSAGE.c:833
  7c:	6ae3      	ldr	r3, [r4, #44]
  7e:	18f3      	adds	r3, r6, r3
  80:	f913 0c01 	ldrsb.w	r0, [r3, #-1]
  84:	f7ff fffe 	bl	0 <GRAPH_WriteChar>
C:\Documents and Settings\jarek\Pulpit\Privet\Magisterka\Programy\1\um0427\FWLib\project/MESSAGE.c:834
  88:	e8bd 81f0 	ldmia.w	sp!, {r4, r5, r6, r7, r8, pc}
	...
Disassembly of section .text.Show:

00000000 <Show>:
Show():
C:\Documents and Settings\jarek\Pulpit\Privet\Magisterka\Programy\1\um0427\FWLib\project/MESSAGE.c:109
   0:	4bba      	ldr	r3, [pc, #744]	(2ec <Show+0x2ec>)
C:\Documents and Settings\jarek\Pulpit\Privet\Magisterka\Programy\1\um0427\FWLib\project/MESSAGE.c:108
   2:	e92d 4177 	stmdb	sp!, {r0, r1, r2, r4, r5, r6, r8, lr}
C:\Documents and Settings\jarek\Pulpit\Privet\Magisterka\Programy\1\um0427\FWLib\project/MESSAGE.c:109
   6:	781b      	ldrb	r3, [r3, #0]
   8:	3b01      	subs	r3, #1
   a:	2b13      	cmp	r3, #19
   c:	f200 85ea 	bhi.w	be4 <Show+0xbe4>
  10:	e8df f013 	tbh	[pc, r3, lsl #1]
  14:	05e80014 	.word	0x05e80014
  18:	012a009a 	.word	0x012a009a
  1c:	013a013a 	.word	0x013a013a
  20:	0176015c 	.word	0x0176015c
  24:	020a0203 	.word	0x020a0203
  28:	02b10210 	.word	0x02b10210
  2c:	03620334 	.word	0x03620334
  30:	03cf03ae 	.word	0x03cf03ae
  34:	04e80491 	.word	0x04e80491
  38:	05d10529 	.word	0x05d10529
C:\Documents and Settings\jarek\Pulpit\Privet\Magisterka\Programy\1\um0427\FWLib\project/MESSAGE.c:114
  3c:	2103      	movs	r1, #3
  3e:	2006      	movs	r0, #6
  40:	f7ff fffe 	bl	0 <GRAPH_TextGoTo>
C:\Documents and Settings\jarek\Pulpit\Privet\Magisterka\Programy\1\um0427\FWLib\project/MESSAGE.c:115
  44:	48aa      	ldr	r0, [pc, #680]	(2ac <printf+0x2ac>)
  46:	f7ff fffe 	bl	0 <printf>
C:\Documents and Settings\jarek\Pulpit\Privet\Magisterka\Programy\1\um0427\FWLib\project/MESSAGE.c:116
  4a:	2104      	movs	r1, #4
  4c:	2006      	movs	r0, #6
  4e:	f7ff fffe 	bl	0 <GRAPH_TextGoTo>
C:\Documents and Settings\jarek\Pulpit\Privet\Magisterka\Programy\1\um0427\FWLib\project/MESSAGE.c:117
  52:	48a7      	ldr	r0, [pc, #668]	(2a0 <printf+0x2a0>)
  54:	f7ff fffe 	bl	0 <printf>
C:\Documents and Settings\jarek\Pulpit\Privet\Magisterka\Programy\1\um0427\FWLib\project/MESSAGE.c:118
  58:	2105      	movs	r1, #5
  5a:	2006      	movs	r0, #6
  5c:	f7ff fffe 	bl	0 <GRAPH_TextGoTo>
C:\Documents and Settings\jarek\Pulpit\Privet\Magisterka\Programy\1\um0427\FWLib\project/MESSAGE.c:119
  60:	48a3      	ldr	r0, [pc, #652]	(290 <printf+0x290>)
  62:	f7ff fffe 	bl	0 <printf>
C:\Documents and Settings\jarek\Pulpit\Privet\Magisterka\Programy\1\um0427\FWLib\project/MESSAGE.c:120
  66:	2006      	movs	r0, #6
  68:	4601      	mov	r1, r0
  6a:	f7ff fffe 	bl	0 <GRAPH_TextGoTo>
C:\Documents and Settings\jarek\Pulpit\Privet\Magisterka\Programy\1\um0427\FWLib\project/MESSAGE.c:121
  6e:	48a0      	ldr	r0, [pc, #640]	(284 <printf+0x284>)
  70:	f7ff fffe 	bl	0 <printf>
C:\Documents and Settings\jarek\Pulpit\Privet\Magisterka\Programy\1\um0427\FWLib\project/MESSAGE.c:122
  74:	2107      	movs	r1, #7
  76:	2006      	movs	r0, #6
  78:	f7ff fffe 	bl	0 <GRAPH_TextGoTo>
C:\Documents and Settings\jarek\Pulpit\Privet\Magisterka\Programy\1\um0427\FWLib\project/MESSAGE.c:123
  7c:	489c      	ldr	r0, [pc, #624]	(274 <printf+0x274>)
  7e:	f7ff fffe 	bl	0 <printf>
C:\Documents and Settings\jarek\Pulpit\Privet\Magisterka\Programy\1\um0427\FWLib\project/MESSAGE.c:124
  82:	2108      	movs	r1, #8
  84:	2006      	movs	r0, #6
  86:	f7ff fffe 	bl	0 <GRAPH_TextGoTo>
C:\Documents and Settings\jarek\Pulpit\Privet\Magisterka\Programy\1\um0427\FWLib\project/MESSAGE.c:125
  8a:	4899      	ldr	r0, [pc, #612]	(268 <printf+0x268>)
  8c:	f7ff fffe 	bl	0 <printf>
C:\Documents and Settings\jarek\Pulpit\Privet\Magisterka\Programy\1\um0427\FWLib\project/MESSAGE.c:126
  90:	2109      	movs	r1, #9
  92:	2006      	movs	r0, #6
  94:	f7ff fffe 	bl	0 <GRAPH_TextGoTo>
C:\Documents and Settings\jarek\Pulpit\Privet\Magisterka\Programy\1\um0427\FWLib\project/MESSAGE.c:127
  98:	4895      	ldr	r0, [pc, #596]	(258 <printf+0x258>)
  9a:	f7ff fffe 	bl	0 <printf>
C:\Documents and Settings\jarek\Pulpit\Privet\Magisterka\Programy\1\um0427\FWLib\project/MESSAGE.c:128
  9e:	210a      	movs	r1, #10
  a0:	2006      	movs	r0, #6
  a2:	f7ff fffe 	bl	0 <GRAPH_TextGoTo>
C:\Documents and Settings\jarek\Pulpit\Privet\Magisterka\Programy\1\um0427\FWLib\project/MESSAGE.c:129
  a6:	4892      	ldr	r0, [pc, #584]	(24c <printf+0x24c>)
  a8:	f7ff fffe 	bl	0 <printf>
C:\Documents and Settings\jarek\Pulpit\Privet\Magisterka\Programy\1\um0427\FWLib\project/MESSAGE.c:131
  ac:	2300      	movs	r3, #0
  ae:	9300      	str	r3, [sp, #0]
  b0:	2024      	movs	r0, #36
  b2:	210f      	movs	r1, #15
  b4:	22a8      	movs	r2, #168
  b6:	334e      	adds	r3, #78
  b8:	f7ff fffe 	bl	0 <GRAPH_RectangleFilled>
C:\Documents and Settings\jarek\Pulpit\Privet\Magisterka\Programy\1\um0427\FWLib\project/MESSAGE.c:132
  bc:	2401      	movs	r4, #1
  be:	210f      	movs	r1, #15
  c0:	22a8      	movs	r2, #168
  c2:	234e      	movs	r3, #78
  c4:	2024      	movs	r0, #36
  c6:	9400      	str	r4, [sp, #0]
  c8:	f7ff fffe 	bl	0 <GRAPH_Rectangle>
C:\Documents and Settings\jarek\Pulpit\Privet\Magisterka\Programy\1\um0427\FWLib\project/MESSAGE.c:133
  cc:	20cc      	movs	r0, #204
  ce:	2110      	movs	r1, #16
  d0:	235d      	movs	r3, #93
  d2:	4602      	mov	r2, r0
  d4:	9400      	str	r4, [sp, #0]
  d6:	f7ff fffe 	bl	0 <GRAPH_Line>
C:\Documents and Settings\jarek\Pulpit\Privet\Magisterka\Programy\1\um0427\FWLib\project/MESSAGE.c:134
  da:	215d      	movs	r1, #93
  dc:	22cc      	movs	r2, #204
  de:	460b      	mov	r3, r1
  e0:	9400      	str	r4, [sp, #0]
  e2:	2025      	movs	r0, #37
C:\Documents and Settings\jarek\Pulpit\Privet\Magisterka\Programy\1\um0427\FWLib\project/MESSAGE.c:137
  e4:	4c83      	ldr	r4, [pc, #524]	(2f4 <Show+0x2f4>)
C:\Documents and Settings\jarek\Pulpit\Privet\Magisterka\Programy\1\um0427\FWLib\project/MESSAGE.c:134
  e6:	f7ff fffe 	bl	0 <GRAPH_Line>
C:\Documents and Settings\jarek\Pulpit\Privet\Magisterka\Programy\1\um0427\FWLib\project/MESSAGE.c:135
  ea:	f7ff fffe 	bl	0 <GRAPH_WhiteBlack>
C:\Documents and Settings\jarek\Pulpit\Privet\Magisterka\Programy\1\um0427\FWLib\project/MESSAGE.c:136
  ee:	2103      	movs	r1, #3
  f0:	2007      	movs	r0, #7
  f2:	f7ff fffe 	bl	0 <GRAPH_TextGoTo>
C:\Documents and Settings\jarek\Pulpit\Privet\Magisterka\Programy\1\um0427\FWLib\project/MESSAGE.c:137
  f6:	6820      	ldr	r0, [r4, #0]
  f8:	f7ff fffe 	bl	0 <printf>
C:\Documents and Settings\jarek\Pulpit\Privet\Magisterka\Programy\1\um0427\FWLib\project/MESSAGE.c:138
  fc:	2104      	movs	r1, #4
  fe:	2007      	movs	r0, #7
 100:	f7ff fffe 	bl	0 <GRAPH_TextGoTo>
C:\Documents and Settings\jarek\Pulpit\Privet\Magisterka\Programy\1\um0427\FWLib\project/MESSAGE.c:139
 104:	6860      	ldr	r0, [r4, #4]
 106:	f7ff fffe 	bl	0 <printf>
C:\Documents and Settings\jarek\Pulpit\Privet\Magisterka\Programy\1\um0427\FWLib\project/MESSAGE.c:140
 10a:	2105      	movs	r1, #5
 10c:	2007      	movs	r0, #7
 10e:	f7ff fffe 	bl	0 <GRAPH_TextGoTo>
C:\Documents and Settings\jarek\Pulpit\Privet\Magisterka\Programy\1\um0427\FWLib\project/MESSAGE.c:141
 112:	68a0      	ldr	r0, [r4, #8]
 114:	f7ff fffe 	bl	0 <printf>
C:\Documents and Settings\jarek\Pulpit\Privet\Magisterka\Programy\1\um0427\FWLib\project/MESSAGE.c:142
 118:	2106      	movs	r1, #6
 11a:	2007      	movs	r0, #7
 11c:	f7ff fffe 	bl	0 <GRAPH_TextGoTo>
C:\Documents and Settings\jarek\Pulpit\Privet\Magisterka\Programy\1\um0427\FWLib\project/MESSAGE.c:143
 120:	68e0      	ldr	r0, [r4, #12]
 122:	f7ff fffe 	bl	0 <printf>
C:\Documents and Settings\jarek\Pulpit\Privet\Magisterka\Programy\1\um0427\FWLib\project/MESSAGE.c:144
 126:	2007      	movs	r0, #7
 128:	4601      	mov	r1, r0
 12a:	f7ff fffe 	bl	0 <GRAPH_TextGoTo>
C:\Documents and Settings\jarek\Pulpit\Privet\Magisterka\Programy\1\um0427\FWLib\project/MESSAGE.c:145
 12e:	6920      	ldr	r0, [r4, #16]
 130:	f7ff fffe 	bl	0 <printf>
C:\Documents and Settings\jarek\Pulpit\Privet\Magisterka\Programy\1\um0427\FWLib\project/MESSAGE.c:146
 134:	2108      	movs	r1, #8
 136:	2007      	movs	r0, #7
 138:	f7ff fffe 	bl	0 <GRAPH_TextGoTo>
C:\Documents and Settings\jarek\Pulpit\Privet\Magisterka\Programy\1\um0427\FWLib\project/MESSAGE.c:147
 13c:	6960      	ldr	r0, [r4, #20]
 13e:	f7ff fffe 	bl	0 <printf>
C:\Documents and Settings\jarek\Pulpit\Privet\Magisterka\Programy\1\um0427\FWLib\project/MESSAGE.c:148
 142:	2202      	movs	r2, #2
 144:	f000 bd4c 	b.w	be0 <Show+0xbe0>
C:\Documents and Settings\jarek\Pulpit\Privet\Magisterka\Programy\1\um0427\FWLib\project/MESSAGE.c:154
 148:	f7ff fffe 	bl	0 <GRAPH_WhiteBlack>
C:\Documents and Settings\jarek\Pulpit\Privet\Magisterka\Programy\1\um0427\FWLib\project/MESSAGE.c:156
 14c:	2103      	movs	r1, #3
 14e:	2006      	movs	r0, #6
 150:	f7ff fffe 	bl	0 <GRAPH_TextGoTo>
C:\Documents and Settings\jarek\Pulpit\Privet\Magisterka\Programy\1\um0427\FWLib\project/MESSAGE.c:157
 154:	4866      	ldr	r0, [pc, #408]	(19c <printf+0x19c>)
 156:	f7ff fffe 	bl	0 <printf>
C:\Documents and Settings\jarek\Pulpit\Privet\Magisterka\Programy\1\um0427\FWLib\project/MESSAGE.c:158
 15a:	2104      	movs	r1, #4
 15c:	2006      	movs	r0, #6
 15e:	f7ff fffe 	bl	0 <GRAPH_TextGoTo>
C:\Documents and Settings\jarek\Pulpit\Privet\Magisterka\Programy\1\um0427\FWLib\project/MESSAGE.c:159
 162:	4863      	ldr	r0, [pc, #396]	(190 <printf+0x190>)
 164:	f7ff fffe 	bl	0 <printf>
C:\Documents and Settings\jarek\Pulpit\Privet\Magisterka\Programy\1\um0427\FWLib\project/MESSAGE.c:160
 168:	2105      	movs	r1, #5
 16a:	2006      	movs	r0, #6
 16c:	f7ff fffe 	bl	0 <GRAPH_TextGoTo>
C:\Documents and Settings\jarek\Pulpit\Privet\Magisterka\Programy\1\um0427\FWLib\project/MESSAGE.c:161
 170:	485f      	ldr	r0, [pc, #380]	(180 <printf+0x180>)
 172:	f7ff fffe 	bl	0 <printf>
C:\Documents and Settings\jarek\Pulpit\Privet\Magisterka\Programy\1\um0427\FWLib\project/MESSAGE.c:162
 176:	2006      	movs	r0, #6
 178:	4601      	mov	r1, r0
 17a:	f7ff fffe 	bl	0 <GRAPH_TextGoTo>
C:\Documents and Settings\jarek\Pulpit\Privet\Magisterka\Programy\1\um0427\FWLib\project/MESSAGE.c:163
 17e:	485c      	ldr	r0, [pc, #368]	(174 <printf+0x174>)
 180:	f7ff fffe 	bl	0 <printf>
C:\Documents and Settings\jarek\Pulpit\Privet\Magisterka\Programy\1\um0427\FWLib\project/MESSAGE.c:164
 184:	2107      	movs	r1, #7
 186:	2006      	movs	r0, #6
 188:	f7ff fffe 	bl	0 <GRAPH_TextGoTo>
C:\Documents and Settings\jarek\Pulpit\Privet\Magisterka\Programy\1\um0427\FWLib\project/MESSAGE.c:165
 18c:	4858      	ldr	r0, [pc, #352]	(164 <printf+0x164>)
 18e:	f7ff fffe 	bl	0 <printf>
C:\Documents and Settings\jarek\Pulpit\Privet\Magisterka\Programy\1\um0427\FWLib\project/MESSAGE.c:166
 192:	2108      	movs	r1, #8
 194:	2006      	movs	r0, #6
 196:	f7ff fffe 	bl	0 <GRAPH_TextGoTo>
C:\Documents and Settings\jarek\Pulpit\Privet\Magisterka\Programy\1\um0427\FWLib\project/MESSAGE.c:167
 19a:	4855      	ldr	r0, [pc, #340]	(158 <printf+0x158>)
 19c:	f7ff fffe 	bl	0 <printf>
C:\Documents and Settings\jarek\Pulpit\Privet\Magisterka\Programy\1\um0427\FWLib\project/MESSAGE.c:168
 1a0:	2109      	movs	r1, #9
 1a2:	2006      	movs	r0, #6
 1a4:	f7ff fffe 	bl	0 <GRAPH_TextGoTo>
C:\Documents and Settings\jarek\Pulpit\Privet\Magisterka\Programy\1\um0427\FWLib\project/MESSAGE.c:169
 1a8:	4851      	ldr	r0, [pc, #324]	(148 <printf+0x148>)
 1aa:	f7ff fffe 	bl	0 <printf>
C:\Documents and Settings\jarek\Pulpit\Privet\Magisterka\Programy\1\um0427\FWLib\project/MESSAGE.c:170
 1ae:	210a      	movs	r1, #10
 1b0:	2006      	movs	r0, #6
 1b2:	f7ff fffe 	bl	0 <GRAPH_TextGoTo>
C:\Documents and Settings\jarek\Pulpit\Privet\Magisterka\Programy\1\um0427\FWLib\project/MESSAGE.c:171
 1b6:	484e      	ldr	r0, [pc, #312]	(13c <printf+0x13c>)
 1b8:	f7ff fffe 	bl	0 <printf>
C:\Documents and Settings\jarek\Pulpit\Privet\Magisterka\Programy\1\um0427\FWLib\project/MESSAGE.c:173
 1bc:	2600      	movs	r6, #0
 1be:	2024      	movs	r0, #36
 1c0:	210f      	movs	r1, #15
 1c2:	22a8      	movs	r2, #168
 1c4:	234e      	movs	r3, #78
C:\Documents and Settings\jarek\Pulpit\Privet\Magisterka\Programy\1\um0427\FWLib\project/MESSAGE.c:174
 1c6:	2501      	movs	r5, #1
C:\Documents and Settings\jarek\Pulpit\Privet\Magisterka\Programy\1\um0427\FWLib\project/MESSAGE.c:173
 1c8:	9600      	str	r6, [sp, #0]
 1ca:	f7ff fffe 	bl	0 <GRAPH_RectangleFilled>
C:\Documents and Settings\jarek\Pulpit\Privet\Magisterka\Programy\1\um0427\FWLib\project/MESSAGE.c:174
 1ce:	210f      	movs	r1, #15
 1d0:	22a8      	movs	r2, #168
 1d2:	234e      	movs	r3, #78
 1d4:	2024      	movs	r0, #36
 1d6:	9500      	str	r5, [sp, #0]
 1d8:	f7ff fffe 	bl	0 <GRAPH_Rectangle>
C:\Documents and Settings\jarek\Pulpit\Privet\Magisterka\Programy\1\um0427\FWLib\project/MESSAGE.c:175
 1dc:	20cc      	movs	r0, #204
 1de:	2110      	movs	r1, #16
 1e0:	235d      	movs	r3, #93
 1e2:	4602      	mov	r2, r0
 1e4:	9500      	str	r5, [sp, #0]
 1e6:	f7ff fffe 	bl	0 <GRAPH_Line>
C:\Documents and Settings\jarek\Pulpit\Privet\Magisterka\Programy\1\um0427\FWLib\project/MESSAGE.c:176
 1ea:	215d      	movs	r1, #93
 1ec:	460b      	mov	r3, r1
 1ee:	22cc      	movs	r2, #204
C:\Documents and Settings\jarek\Pulpit\Privet\Magisterka\Programy\1\um0427\FWLib\project/MESSAGE.c:178
 1f0:	4c40      	ldr	r4, [pc, #256]	(2f4 <Show+0x2f4>)
C:\Documents and Settings\jarek\Pulpit\Privet\Magisterka\Programy\1\um0427\FWLib\project/MESSAGE.c:176
 1f2:	2025      	movs	r0, #37
 1f4:	9500      	str	r5, [sp, #0]
 1f6:	f7ff fffe 	bl	0 <GRAPH_Line>
C:\Documents and Settings\jarek\Pulpit\Privet\Magisterka\Programy\1\um0427\FWLib\project/MESSAGE.c:177
 1fa:	2103      	movs	r1, #3
 1fc:	2007      	movs	r0, #7
 1fe:	f7ff fffe 	bl	0 <GRAPH_TextGoTo>
C:\Documents and Settings\jarek\Pulpit\Privet\Magisterka\Programy\1\um0427\FWLib\project/MESSAGE.c:178
 202:	6820      	ldr	r0, [r4, #0]
 204:	f7ff fffe 	bl	0 <printf>
C:\Documents and Settings\jarek\Pulpit\Privet\Magisterka\Programy\1\um0427\FWLib\project/MESSAGE.c:179
 208:	2104      	movs	r1, #4
 20a:	2007      	movs	r0, #7
 20c:	f7ff fffe 	bl	0 <GRAPH_TextGoTo>
C:\Documents and Settings\jarek\Pulpit\Privet\Magisterka\Programy\1\um0427\FWLib\project/MESSAGE.c:180
 210:	6860      	ldr	r0, [r4, #4]
 212:	f7ff fffe 	bl	0 <printf>
C:\Documents and Settings\jarek\Pulpit\Privet\Magisterka\Programy\1\um0427\FWLib\project/MESSAGE.c:181
 216:	2105      	movs	r1, #5
 218:	2007      	movs	r0, #7
 21a:	f7ff fffe 	bl	0 <GRAPH_TextGoTo>
C:\Documents and Settings\jarek\Pulpit\Privet\Magisterka\Programy\1\um0427\FWLib\project/MESSAGE.c:182
 21e:	68a0      	ldr	r0, [r4, #8]
 220:	f7ff fffe 	bl	0 <printf>
C:\Documents and Settings\jarek\Pulpit\Privet\Magisterka\Programy\1\um0427\FWLib\project/MESSAGE.c:183
 224:	2106      	movs	r1, #6
 226:	2007      	movs	r0, #7
 228:	f7ff fffe 	bl	0 <GRAPH_TextGoTo>
C:\Documents and Settings\jarek\Pulpit\Privet\Magisterka\Programy\1\um0427\FWLib\project/MESSAGE.c:184
 22c:	68e0      	ldr	r0, [r4, #12]
 22e:	f7ff fffe 	bl	0 <printf>
C:\Documents and Settings\jarek\Pulpit\Privet\Magisterka\Programy\1\um0427\FWLib\project/MESSAGE.c:185
 232:	2007      	movs	r0, #7
 234:	4601      	mov	r1, r0
 236:	f7ff fffe 	bl	0 <GRAPH_TextGoTo>
C:\Documents and Settings\jarek\Pulpit\Privet\Magisterka\Programy\1\um0427\FWLib\project/MESSAGE.c:186
 23a:	6920      	ldr	r0, [r4, #16]
 23c:	f7ff fffe 	bl	0 <printf>
C:\Documents and Settings\jarek\Pulpit\Privet\Magisterka\Programy\1\um0427\FWLib\project/MESSAGE.c:187
 240:	2108      	movs	r1, #8
 242:	2007      	movs	r0, #7
 244:	f7ff fffe 	bl	0 <GRAPH_TextGoTo>
C:\Documents and Settings\jarek\Pulpit\Privet\Magisterka\Programy\1\um0427\FWLib\project/MESSAGE.c:188
 248:	6960      	ldr	r0, [r4, #20]
 24a:	f7ff fffe 	bl	0 <printf>
C:\Documents and Settings\jarek\Pulpit\Privet\Magisterka\Programy\1\um0427\FWLib\project/MESSAGE.c:190
 24e:	200e      	movs	r0, #14
 250:	210a      	movs	r1, #10
 252:	4a29      	ldr	r2, [pc, #164]	(2f8 <Show+0x2f8>)
 254:	4633      	mov	r3, r6
C:\Documents and Settings\jarek\Pulpit\Privet\Magisterka\Programy\1\um0427\FWLib\project/MESSAGE.c:189
 256:	f884 5075 	strb.w	r5, [r4, #117]
C:\Documents and Settings\jarek\Pulpit\Privet\Magisterka\Programy\1\um0427\FWLib\project/MESSAGE.c:190
 25a:	f7ff fffe 	bl	0 <Show>
C:\Documents and Settings\jarek\Pulpit\Privet\Magisterka\Programy\1\um0427\FWLib\project/MESSAGE.c:191
 25e:	2015      	movs	r0, #21
 260:	210a      	movs	r1, #10
 262:	4a26      	ldr	r2, [pc, #152]	(2fc <Show+0x2fc>)
 264:	462b      	mov	r3, r5
 266:	e02c      	b.n	2c2 <Show+0x2c2>
C:\Documents and Settings\jarek\Pulpit\Privet\Magisterka\Programy\1\um0427\FWLib\project/MESSAGE.c:195
 268:	f7ff fffe 	bl	0 <KEY_CheckKey>
 26c:	2802      	cmp	r0, #2
 26e:	d005      	beq.n	27c <Show+0x27c>
 270:	2804      	cmp	r0, #4
 272:	d005      	beq.n	280 <Show+0x280>
 274:	2801      	cmp	r0, #1
 276:	d005      	beq.n	284 <Show+0x284>
 278:	f000 bcb4 	b.w	be4 <Show+0xbe4>
C:\Documents and Settings\jarek\Pulpit\Privet\Magisterka\Programy\1\um0427\FWLib\project/MESSAGE.c:197
 27c:	2206      	movs	r2, #6
 27e:	e370      	b.n	962 <Show+0x962>
C:\Documents and Settings\jarek\Pulpit\Privet\Magisterka\Programy\1\um0427\FWLib\project/MESSAGE.c:201
 280:	2205      	movs	r2, #5
 282:	e36e      	b.n	962 <Show+0x962>
C:\Documents and Settings\jarek\Pulpit\Privet\Magisterka\Programy\1\um0427\FWLib\project/MESSAGE.c:205
 284:	2207      	movs	r2, #7
 286:	e36c      	b.n	962 <Show+0x962>
C:\Documents and Settings\jarek\Pulpit\Privet\Magisterka\Programy\1\um0427\FWLib\project/MESSAGE.c:223
 288:	4a1a      	ldr	r2, [pc, #104]	(2f4 <Show+0x2f4>)
 28a:	f892 3075 	ldrb.w	r3, [r2, #117]
 28e:	b963      	cbnz	r3, 2aa <Show+0x2aa>
C:\Documents and Settings\jarek\Pulpit\Privet\Magisterka\Programy\1\um0427\FWLib\project/MESSAGE.c:224
 290:	2401      	movs	r4, #1
 292:	f882 4075 	strb.w	r4, [r2, #117]
C:\Documents and Settings\jarek\Pulpit\Privet\Magisterka\Programy\1\um0427\FWLib\project/MESSAGE.c:225
 296:	200e      	movs	r0, #14
 298:	210a      	movs	r1, #10
 29a:	4a17      	ldr	r2, [pc, #92]	(2f8 <Show+0x2f8>)
 29c:	f7ff fffe 	bl	0 <Show>
C:\Documents and Settings\jarek\Pulpit\Privet\Magisterka\Programy\1\um0427\FWLib\project/MESSAGE.c:226
 2a0:	2015      	movs	r0, #21
 2a2:	210a      	movs	r1, #10
 2a4:	4a15      	ldr	r2, [pc, #84]	(2fc <Show+0x2fc>)
 2a6:	4623      	mov	r3, r4
 2a8:	e00b      	b.n	2c2 <Show+0x2c2>
C:\Documents and Settings\jarek\Pulpit\Privet\Magisterka\Programy\1\um0427\FWLib\project/MESSAGE.c:228
 2aa:	2300      	movs	r3, #0
 2ac:	f882 3075 	strb.w	r3, [r2, #117]
C:\Documents and Settings\jarek\Pulpit\Privet\Magisterka\Programy\1\um0427\FWLib\project/MESSAGE.c:229
 2b0:	2015      	movs	r0, #21
 2b2:	210a      	movs	r1, #10
 2b4:	4a11      	ldr	r2, [pc, #68]	(2fc <Show+0x2fc>)
 2b6:	f7ff fffe 	bl	0 <Show>
C:\Documents and Settings\jarek\Pulpit\Privet\Magisterka\Programy\1\um0427\FWLib\project/MESSAGE.c:230
 2ba:	4a0f      	ldr	r2, [pc, #60]	(2f8 <Show+0x2f8>)
 2bc:	200e      	movs	r0, #14
 2be:	210a      	movs	r1, #10
 2c0:	2301      	movs	r3, #1
 2c2:	f7ff fffe 	bl	0 <Show>
C:\Documents and Settings\jarek\Pulpit\Privet\Magisterka\Programy\1\um0427\FWLib\project/MESSAGE.c:232
 2c6:	2204      	movs	r2, #4
 2c8:	f000 bc8a 	b.w	be0 <Show+0xbe0>
C:\Documents and Settings\jarek\Pulpit\Privet\Magisterka\Programy\1\um0427\FWLib\project/MESSAGE.c:235
 2cc:	4909      	ldr	r1, [pc, #36]	(2f4 <Show+0x2f4>)
 2ce:	f891 3075 	ldrb.w	r3, [r1, #117]
 2d2:	2b01      	cmp	r3, #1
 2d4:	d104      	bne.n	2e0 <Show+0x2e0>
C:\Documents and Settings\jarek\Pulpit\Privet\Magisterka\Programy\1\um0427\FWLib\project/MESSAGE.c:236
 2d6:	698b      	ldr	r3, [r1, #24]
 2d8:	69ca      	ldr	r2, [r1, #28]
 2da:	601a      	str	r2, [r3, #0]
 2dc:	f000 bc7d 	b.w	bda <Show+0xbda>
C:\Documents and Settings\jarek\Pulpit\Privet\Magisterka\Programy\1\um0427\FWLib\project/MESSAGE.c:239
 2e0:	698b      	ldr	r3, [r1, #24]
 2e2:	6a0a      	ldr	r2, [r1, #32]
 2e4:	601a      	str	r2, [r3, #0]
 2e6:	f000 bc71 	b.w	bcc <Show+0xbcc>
 2ea:	46c0      	nop			(mov r8, r8)
 2ec:	00000000 	.word	0x00000000
 2f0:	00000028 	.word	0x00000028
 2f4:	00000000 	.word	0x00000000
 2f8:	00000045 	.word	0x00000045
 2fc:	00000049 	.word	0x00000049
C:\Documents and Settings\jarek\Pulpit\Privet\Magisterka\Programy\1\um0427\FWLib\project/MESSAGE.c:248
 300:	2103      	movs	r1, #3
 302:	2006      	movs	r0, #6
 304:	f7ff fffe 	bl	0 <GRAPH_TextGoTo>
C:\Documents and Settings\jarek\Pulpit\Privet\Magisterka\Programy\1\um0427\FWLib\project/MESSAGE.c:249
 308:	48c3      	ldr	r0, [pc, #780]	(310 <printf+0x310>)
 30a:	f7ff fffe 	bl	0 <printf>
C:\Documents and Settings\jarek\Pulpit\Privet\Magisterka\Programy\1\um0427\FWLib\project/MESSAGE.c:250
 30e:	2104      	movs	r1, #4
 310:	2006      	movs	r0, #6
 312:	f7ff fffe 	bl	0 <GRAPH_TextGoTo>
C:\Documents and Settings\jarek\Pulpit\Privet\Magisterka\Programy\1\um0427\FWLib\project/MESSAGE.c:251
 316:	48c0      	ldr	r0, [pc, #768]	(304 <printf+0x304>)
 318:	f7ff fffe 	bl	0 <printf>
C:\Documents and Settings\jarek\Pulpit\Privet\Magisterka\Programy\1\um0427\FWLib\project/MESSAGE.c:252
 31c:	2105      	movs	r1, #5
 31e:	2006      	movs	r0, #6
 320:	f7ff fffe 	bl	0 <GRAPH_TextGoTo>
C:\Documents and Settings\jarek\Pulpit\Privet\Magisterka\Programy\1\um0427\FWLib\project/MESSAGE.c:253
 324:	48bc      	ldr	r0, [pc, #752]	(2f4 <printf+0x2f4>)
 326:	f7ff fffe 	bl	0 <printf>
C:\Documents and Settings\jarek\Pulpit\Privet\Magisterka\Programy\1\um0427\FWLib\project/MESSAGE.c:254
 32a:	2006      	movs	r0, #6
 32c:	4601      	mov	r1, r0
 32e:	f7ff fffe 	bl	0 <GRAPH_TextGoTo>
C:\Documents and Settings\jarek\Pulpit\Privet\Magisterka\Programy\1\um0427\FWLib\project/MESSAGE.c:255
 332:	48b9      	ldr	r0, [pc, #740]	(2e8 <printf+0x2e8>)
 334:	f7ff fffe 	bl	0 <printf>
C:\Documents and Settings\jarek\Pulpit\Privet\Magisterka\Programy\1\um0427\FWLib\project/MESSAGE.c:256
 338:	2107      	movs	r1, #7
 33a:	2006      	movs	r0, #6
 33c:	f7ff fffe 	bl	0 <GRAPH_TextGoTo>
C:\Documents and Settings\jarek\Pulpit\Privet\Magisterka\Programy\1\um0427\FWLib\project/MESSAGE.c:257
 340:	48b5      	ldr	r0, [pc, #724]	(2d8 <printf+0x2d8>)
 342:	f7ff fffe 	bl	0 <printf>
C:\Documents and Settings\jarek\Pulpit\Privet\Magisterka\Programy\1\um0427\FWLib\project/MESSAGE.c:258
 346:	2108      	movs	r1, #8
 348:	2006      	movs	r0, #6
 34a:	f7ff fffe 	bl	0 <GRAPH_TextGoTo>
C:\Documents and Settings\jarek\Pulpit\Privet\Magisterka\Programy\1\um0427\FWLib\project/MESSAGE.c:259
 34e:	48b2      	ldr	r0, [pc, #712]	(2cc <printf+0x2cc>)
 350:	f7ff fffe 	bl	0 <printf>
C:\Documents and Settings\jarek\Pulpit\Privet\Magisterka\Programy\1\um0427\FWLib\project/MESSAGE.c:260
 354:	2109      	movs	r1, #9
 356:	2006      	movs	r0, #6
 358:	f7ff fffe 	bl	0 <GRAPH_TextGoTo>
C:\Documents and Settings\jarek\Pulpit\Privet\Magisterka\Programy\1\um0427\FWLib\project/MESSAGE.c:261
 35c:	48ae      	ldr	r0, [pc, #696]	(2bc <printf+0x2bc>)
 35e:	f7ff fffe 	bl	0 <printf>
C:\Documents and Settings\jarek\Pulpit\Privet\Magisterka\Programy\1\um0427\FWLib\project/MESSAGE.c:262
 362:	210a      	movs	r1, #10
 364:	2006      	movs	r0, #6
 366:	f7ff fffe 	bl	0 <GRAPH_TextGoTo>
C:\Documents and Settings\jarek\Pulpit\Privet\Magisterka\Programy\1\um0427\FWLib\project/MESSAGE.c:263
 36a:	48ab      	ldr	r0, [pc, #684]	(2b0 <printf+0x2b0>)
 36c:	f7ff fffe 	bl	0 <printf>
C:\Documents and Settings\jarek\Pulpit\Privet\Magisterka\Programy\1\um0427\FWLib\project/MESSAGE.c:265
 370:	2300      	movs	r3, #0
 372:	9300      	str	r3, [sp, #0]
 374:	2024      	movs	r0, #36
 376:	210f      	movs	r1, #15
 378:	22a8      	movs	r2, #168
 37a:	334e      	adds	r3, #78
 37c:	f7ff fffe 	bl	0 <GRAPH_RectangleFilled>
C:\Documents and Settings\jarek\Pulpit\Privet\Magisterka\Programy\1\um0427\FWLib\project/MESSAGE.c:267
 380:	2501      	movs	r5, #1
 382:	210f      	movs	r1, #15
 384:	22a8      	movs	r2, #168
 386:	234e      	movs	r3, #78
 388:	2024      	movs	r0, #36
 38a:	9500      	str	r5, [sp, #0]
 38c:	f7ff fffe 	bl	0 <GRAPH_Rectangle>
C:\Documents and Settings\jarek\Pulpit\Privet\Magisterka\Programy\1\um0427\FWLib\project/MESSAGE.c:268
 390:	20cc      	movs	r0, #204
 392:	2110      	movs	r1, #16
 394:	235d      	movs	r3, #93
 396:	4602      	mov	r2, r0
 398:	9500      	str	r5, [sp, #0]
 39a:	f7ff fffe 	bl	0 <GRAPH_Line>
C:\Documents and Settings\jarek\Pulpit\Privet\Magisterka\Programy\1\um0427\FWLib\project/MESSAGE.c:269
 39e:	215d      	movs	r1, #93
 3a0:	460b      	mov	r3, r1
 3a2:	22cc      	movs	r2, #204
C:\Documents and Settings\jarek\Pulpit\Privet\Magisterka\Programy\1\um0427\FWLib\project/MESSAGE.c:272
 3a4:	4c9d      	ldr	r4, [pc, #628]	(61c <Show+0x61c>)
C:\Documents and Settings\jarek\Pulpit\Privet\Magisterka\Programy\1\um0427\FWLib\project/MESSAGE.c:269
 3a6:	2025      	movs	r0, #37
 3a8:	9500      	str	r5, [sp, #0]
 3aa:	f7ff fffe 	bl	0 <GRAPH_Line>
C:\Documents and Settings\jarek\Pulpit\Privet\Magisterka\Programy\1\um0427\FWLib\project/MESSAGE.c:270
 3ae:	f7ff fffe 	bl	0 <GRAPH_WhiteBlack>
C:\Documents and Settings\jarek\Pulpit\Privet\Magisterka\Programy\1\um0427\FWLib\project/MESSAGE.c:271
 3b2:	2103      	movs	r1, #3
 3b4:	2007      	movs	r0, #7
 3b6:	f7ff fffe 	bl	0 <GRAPH_TextGoTo>
C:\Documents and Settings\jarek\Pulpit\Privet\Magisterka\Programy\1\um0427\FWLib\project/MESSAGE.c:272
 3ba:	6820      	ldr	r0, [r4, #0]
 3bc:	f7ff fffe 	bl	0 <printf>
C:\Documents and Settings\jarek\Pulpit\Privet\Magisterka\Programy\1\um0427\FWLib\project/MESSAGE.c:273
 3c0:	2104      	movs	r1, #4
 3c2:	2007      	movs	r0, #7
 3c4:	f7ff fffe 	bl	0 <GRAPH_TextGoTo>
C:\Documents and Settings\jarek\Pulpit\Privet\Magisterka\Programy\1\um0427\FWLib\project/MESSAGE.c:274
 3c8:	6860      	ldr	r0, [r4, #4]
 3ca:	f7ff fffe 	bl	0 <printf>
C:\Documents and Settings\jarek\Pulpit\Privet\Magisterka\Programy\1\um0427\FWLib\project/MESSAGE.c:275
 3ce:	2105      	movs	r1, #5
 3d0:	2007      	movs	r0, #7
 3d2:	f7ff fffe 	bl	0 <GRAPH_TextGoTo>
C:\Documents and Settings\jarek\Pulpit\Privet\Magisterka\Programy\1\um0427\FWLib\project/MESSAGE.c:276
 3d6:	68a0      	ldr	r0, [r4, #8]
 3d8:	f7ff fffe 	bl	0 <printf>
C:\Documents and Settings\jarek\Pulpit\Privet\Magisterka\Programy\1\um0427\FWLib\project/MESSAGE.c:277
 3dc:	2106      	movs	r1, #6
 3de:	2007      	movs	r0, #7
 3e0:	f7ff fffe 	bl	0 <GRAPH_TextGoTo>
C:\Documents and Settings\jarek\Pulpit\Privet\Magisterka\Programy\1\um0427\FWLib\project/MESSAGE.c:278
 3e4:	68e0      	ldr	r0, [r4, #12]
 3e6:	f7ff fffe 	bl	0 <printf>
C:\Documents and Settings\jarek\Pulpit\Privet\Magisterka\Programy\1\um0427\FWLib\project/MESSAGE.c:279
 3ea:	2007      	movs	r0, #7
 3ec:	4601      	mov	r1, r0
 3ee:	f7ff fffe 	bl	0 <GRAPH_TextGoTo>
C:\Documents and Settings\jarek\Pulpit\Privet\Magisterka\Programy\1\um0427\FWLib\project/MESSAGE.c:280
 3f2:	6920      	ldr	r0, [r4, #16]
 3f4:	f7ff fffe 	bl	0 <printf>
C:\Documents and Settings\jarek\Pulpit\Privet\Magisterka\Programy\1\um0427\FWLib\project/MESSAGE.c:281
 3f8:	2108      	movs	r1, #8
 3fa:	2007      	movs	r0, #7
 3fc:	f7ff fffe 	bl	0 <GRAPH_TextGoTo>
C:\Documents and Settings\jarek\Pulpit\Privet\Magisterka\Programy\1\um0427\FWLib\project/MESSAGE.c:282
 400:	6960      	ldr	r0, [r4, #20]
 402:	f7ff fffe 	bl	0 <printf>
C:\Documents and Settings\jarek\Pulpit\Privet\Magisterka\Programy\1\um0427\FWLib\project/MESSAGE.c:284
 406:	4a86      	ldr	r2, [pc, #536]	(620 <Show+0x620>)
C:\Documents and Settings\jarek\Pulpit\Privet\Magisterka\Programy\1\um0427\FWLib\project/MESSAGE.c:283
 408:	f884 5075 	strb.w	r5, [r4, #117]
C:\Documents and Settings\jarek\Pulpit\Privet\Magisterka\Programy\1\um0427\FWLib\project/MESSAGE.c:284
 40c:	2012      	movs	r0, #18
 40e:	210a      	movs	r1, #10
 410:	462b      	mov	r3, r5
 412:	f7ff fffe 	bl	0 <Show>
C:\Documents and Settings\jarek\Pulpit\Privet\Magisterka\Programy\1\um0427\FWLib\project/MESSAGE.c:285
 416:	2209      	movs	r2, #9
 418:	e3e2      	b.n	be0 <Show+0xbe0>
C:\Documents and Settings\jarek\Pulpit\Privet\Magisterka\Programy\1\um0427\FWLib\project/MESSAGE.c:288
 41a:	f7ff fffe 	bl	0 <KEY_CheckKey>
 41e:	2801      	cmp	r0, #1
 420:	f040 83e0 	bne.w	be4 <Show+0xbe4>
C:\Documents and Settings\jarek\Pulpit\Privet\Magisterka\Programy\1\um0427\FWLib\project/MESSAGE.c:290
 424:	220a      	movs	r2, #10
 426:	e29c      	b.n	962 <Show+0x962>
C:\Documents and Settings\jarek\Pulpit\Privet\Magisterka\Programy\1\um0427\FWLib\project/MESSAGE.c:296
 428:	4b7c      	ldr	r3, [pc, #496]	(61c <Show+0x61c>)
 42a:	6999      	ldr	r1, [r3, #24]
 42c:	6a5a      	ldr	r2, [r3, #36]
C:\Documents and Settings\jarek\Pulpit\Privet\Magisterka\Programy\1\um0427\FWLib\project/MESSAGE.c:297
 42e:	6b9b      	ldr	r3, [r3, #56]
C:\Documents and Settings\jarek\Pulpit\Privet\Magisterka\Programy\1\um0427\FWLib\project/MESSAGE.c:296
 430:	600a      	str	r2, [r1, #0]
 432:	e3cc      	b.n	bce <Show+0xbce>
C:\Documents and Settings\jarek\Pulpit\Privet\Magisterka\Programy\1\um0427\FWLib\project/MESSAGE.c:303
 434:	f7ff fffe 	bl	0 <GRAPH_WhiteBlack>
C:\Documents and Settings\jarek\Pulpit\Privet\Magisterka\Programy\1\um0427\FWLib\project/MESSAGE.c:304
 438:	2103      	movs	r1, #3
 43a:	2006      	movs	r0, #6
 43c:	f7ff fffe 	bl	0 <GRAPH_TextGoTo>
C:\Documents and Settings\jarek\Pulpit\Privet\Magisterka\Programy\1\um0427\FWLib\project/MESSAGE.c:305
 440:	4875      	ldr	r0, [pc, #468]	(1d8 <printf+0x1d8>)
 442:	f7ff fffe 	bl	0 <printf>
C:\Documents and Settings\jarek\Pulpit\Privet\Magisterka\Programy\1\um0427\FWLib\project/MESSAGE.c:306
 446:	2104      	movs	r1, #4
 448:	2006      	movs	r0, #6
 44a:	f7ff fffe 	bl	0 <GRAPH_TextGoTo>
C:\Documents and Settings\jarek\Pulpit\Privet\Magisterka\Programy\1\um0427\FWLib\project/MESSAGE.c:307
 44e:	4872      	ldr	r0, [pc, #456]	(1cc <printf+0x1cc>)
 450:	f7ff fffe 	bl	0 <printf>
C:\Documents and Settings\jarek\Pulpit\Privet\Magisterka\Programy\1\um0427\FWLib\project/MESSAGE.c:308
 454:	2105      	movs	r1, #5
 456:	2006      	movs	r0, #6
 458:	f7ff fffe 	bl	0 <GRAPH_TextGoTo>
C:\Documents and Settings\jarek\Pulpit\Privet\Magisterka\Programy\1\um0427\FWLib\project/MESSAGE.c:309
 45c:	486e      	ldr	r0, [pc, #440]	(1bc <printf+0x1bc>)
 45e:	f7ff fffe 	bl	0 <printf>
C:\Documents and Settings\jarek\Pulpit\Privet\Magisterka\Programy\1\um0427\FWLib\project/MESSAGE.c:310
 462:	2006      	movs	r0, #6
 464:	4601      	mov	r1, r0
 466:	f7ff fffe 	bl	0 <GRAPH_TextGoTo>
C:\Documents and Settings\jarek\Pulpit\Privet\Magisterka\Programy\1\um0427\FWLib\project/MESSAGE.c:311
 46a:	486b      	ldr	r0, [pc, #428]	(1b0 <printf+0x1b0>)
 46c:	f7ff fffe 	bl	0 <printf>
C:\Documents and Settings\jarek\Pulpit\Privet\Magisterka\Programy\1\um0427\FWLib\project/MESSAGE.c:312
 470:	2107      	movs	r1, #7
 472:	2006      	movs	r0, #6
 474:	f7ff fffe 	bl	0 <GRAPH_TextGoTo>
C:\Documents and Settings\jarek\Pulpit\Privet\Magisterka\Programy\1\um0427\FWLib\project/MESSAGE.c:313
 478:	4867      	ldr	r0, [pc, #412]	(1a0 <printf+0x1a0>)
 47a:	f7ff fffe 	bl	0 <printf>
C:\Documents and Settings\jarek\Pulpit\Privet\Magisterka\Programy\1\um0427\FWLib\project/MESSAGE.c:314
 47e:	2108      	movs	r1, #8
 480:	2006      	movs	r0, #6
 482:	f7ff fffe 	bl	0 <GRAPH_TextGoTo>
C:\Documents and Settings\jarek\Pulpit\Privet\Magisterka\Programy\1\um0427\FWLib\project/MESSAGE.c:315
 486:	4864      	ldr	r0, [pc, #400]	(194 <printf+0x194>)
 488:	f7ff fffe 	bl	0 <printf>
C:\Documents and Settings\jarek\Pulpit\Privet\Magisterka\Programy\1\um0427\FWLib\project/MESSAGE.c:316
 48c:	2109      	movs	r1, #9
 48e:	2006      	movs	r0, #6
 490:	f7ff fffe 	bl	0 <GRAPH_TextGoTo>
C:\Documents and Settings\jarek\Pulpit\Privet\Magisterka\Programy\1\um0427\FWLib\project/MESSAGE.c:317
 494:	4860      	ldr	r0, [pc, #384]	(184 <printf+0x184>)
 496:	f7ff fffe 	bl	0 <printf>
C:\Documents and Settings\jarek\Pulpit\Privet\Magisterka\Programy\1\um0427\FWLib\project/MESSAGE.c:318
 49a:	210a      	movs	r1, #10
 49c:	2006      	movs	r0, #6
 49e:	f7ff fffe 	bl	0 <GRAPH_TextGoTo>
C:\Documents and Settings\jarek\Pulpit\Privet\Magisterka\Programy\1\um0427\FWLib\project/MESSAGE.c:319
 4a2:	485d      	ldr	r0, [pc, #372]	(178 <printf+0x178>)
 4a4:	f7ff fffe 	bl	0 <printf>
C:\Documents and Settings\jarek\Pulpit\Privet\Magisterka\Programy\1\um0427\FWLib\project/MESSAGE.c:321
 4a8:	f04f 0800 	mov.w	r8, #0	; 0x0
 4ac:	2024      	movs	r0, #36
 4ae:	210f      	movs	r1, #15
 4b0:	22a8      	movs	r2, #168
 4b2:	234e      	movs	r3, #78
C:\Documents and Settings\jarek\Pulpit\Privet\Magisterka\Programy\1\um0427\FWLib\project/MESSAGE.c:322
 4b4:	2601      	movs	r6, #1
C:\Documents and Settings\jarek\Pulpit\Privet\Magisterka\Programy\1\um0427\FWLib\project/MESSAGE.c:321
 4b6:	f8cd 8000 	str.w	r8, [sp]
 4ba:	f7ff fffe 	bl	0 <GRAPH_RectangleFilled>
C:\Documents and Settings\jarek\Pulpit\Privet\Magisterka\Programy\1\um0427\FWLib\project/MESSAGE.c:322
 4be:	210f      	movs	r1, #15
 4c0:	22a8      	movs	r2, #168
 4c2:	234e      	movs	r3, #78
 4c4:	2024      	movs	r0, #36
 4c6:	9600      	str	r6, [sp, #0]
 4c8:	f7ff fffe 	bl	0 <GRAPH_Rectangle>
C:\Documents and Settings\jarek\Pulpit\Privet\Magisterka\Programy\1\um0427\FWLib\project/MESSAGE.c:323
 4cc:	20cc      	movs	r0, #204
 4ce:	2110      	movs	r1, #16
 4d0:	235d      	movs	r3, #93
 4d2:	4602      	mov	r2, r0
 4d4:	9600      	str	r6, [sp, #0]
 4d6:	f7ff fffe 	bl	0 <GRAPH_Line>
C:\Documents and Settings\jarek\Pulpit\Privet\Magisterka\Programy\1\um0427\FWLib\project/MESSAGE.c:324
 4da:	215d      	movs	r1, #93
 4dc:	460b      	mov	r3, r1
 4de:	22cc      	movs	r2, #204
C:\Documents and Settings\jarek\Pulpit\Privet\Magisterka\Programy\1\um0427\FWLib\project/MESSAGE.c:327
 4e0:	4c4e      	ldr	r4, [pc, #312]	(61c <Show+0x61c>)
C:\Documents and Settings\jarek\Pulpit\Privet\Magisterka\Programy\1\um0427\FWLib\project/MESSAGE.c:324
 4e2:	2025      	movs	r0, #37
 4e4:	9600      	str	r6, [sp, #0]
 4e6:	f7ff fffe 	bl	0 <GRAPH_Line>
C:\Documents and Settings\jarek\Pulpit\Privet\Magisterka\Programy\1\um0427\FWLib\project/MESSAGE.c:326
 4ea:	2103      	movs	r1, #3
 4ec:	2007      	movs	r0, #7
 4ee:	f7ff fffe 	bl	0 <GRAPH_TextGoTo>
C:\Documents and Settings\jarek\Pulpit\Privet\Magisterka\Programy\1\um0427\FWLib\project/MESSAGE.c:327
 4f2:	6820      	ldr	r0, [r4, #0]
 4f4:	f7ff fffe 	bl	0 <printf>
C:\Documents and Settings\jarek\Pulpit\Privet\Magisterka\Programy\1\um0427\FWLib\project/MESSAGE.c:329
 4f8:	2104      	movs	r1, #4
 4fa:	2007      	movs	r0, #7
 4fc:	f7ff fffe 	bl	0 <GRAPH_TextGoTo>
C:\Documents and Settings\jarek\Pulpit\Privet\Magisterka\Programy\1\um0427\FWLib\project/MESSAGE.c:330
 500:	6860      	ldr	r0, [r4, #4]
 502:	f7ff fffe 	bl	0 <printf>
C:\Documents and Settings\jarek\Pulpit\Privet\Magisterka\Programy\1\um0427\FWLib\project/MESSAGE.c:332
 506:	2105      	movs	r1, #5
 508:	2007      	movs	r0, #7
 50a:	f7ff fffe 	bl	0 <GRAPH_TextGoTo>
C:\Documents and Settings\jarek\Pulpit\Privet\Magisterka\Programy\1\um0427\FWLib\project/MESSAGE.c:333
 50e:	68a0      	ldr	r0, [r4, #8]
 510:	f7ff fffe 	bl	0 <printf>
C:\Documents and Settings\jarek\Pulpit\Privet\Magisterka\Programy\1\um0427\FWLib\project/MESSAGE.c:335
 514:	2106      	movs	r1, #6
 516:	2007      	movs	r0, #7
 518:	f7ff fffe 	bl	0 <GRAPH_TextGoTo>
C:\Documents and Settings\jarek\Pulpit\Privet\Magisterka\Programy\1\um0427\FWLib\project/MESSAGE.c:336
 51c:	68e0      	ldr	r0, [r4, #12]
 51e:	f7ff fffe 	bl	0 <printf>
C:\Documents and Settings\jarek\Pulpit\Privet\Magisterka\Programy\1\um0427\FWLib\project/MESSAGE.c:338
 522:	2007      	movs	r0, #7
 524:	4601      	mov	r1, r0
 526:	f7ff fffe 	bl	0 <GRAPH_TextGoTo>
C:\Documents and Settings\jarek\Pulpit\Privet\Magisterka\Programy\1\um0427\FWLib\project/MESSAGE.c:339
 52a:	6920      	ldr	r0, [r4, #16]
 52c:	f7ff fffe 	bl	0 <printf>
C:\Documents and Settings\jarek\Pulpit\Privet\Magisterka\Programy\1\um0427\FWLib\project/MESSAGE.c:341
 530:	2108      	movs	r1, #8
 532:	2007      	movs	r0, #7
 534:	f7ff fffe 	bl	0 <GRAPH_TextGoTo>
C:\Documents and Settings\jarek\Pulpit\Privet\Magisterka\Programy\1\um0427\FWLib\project/MESSAGE.c:342
 538:	6960      	ldr	r0, [r4, #20]
 53a:	f7ff fffe 	bl	0 <printf>
C:\Documents and Settings\jarek\Pulpit\Privet\Magisterka\Programy\1\um0427\FWLib\project/MESSAGE.c:344
 53e:	2303      	movs	r3, #3
 540:	f884 3075 	strb.w	r3, [r4, #117]
C:\Documents and Settings\jarek\Pulpit\Privet\Magisterka\Programy\1\um0427\FWLib\project/MESSAGE.c:345
 544:	6aa3      	ldr	r3, [r4, #40]
 546:	4d37      	ldr	r5, [pc, #220]	(624 <Show+0x624>)
 548:	681b      	ldr	r3, [r3, #0]
C:\Documents and Settings\jarek\Pulpit\Privet\Magisterka\Programy\1\um0427\FWLib\project/MESSAGE.c:346
 54a:	2009      	movs	r0, #9
C:\Documents and Settings\jarek\Pulpit\Privet\Magisterka\Programy\1\um0427\FWLib\project/MESSAGE.c:345
 54c:	60ab      	str	r3, [r5, #8]
C:\Documents and Settings\jarek\Pulpit\Privet\Magisterka\Programy\1\um0427\FWLib\project/MESSAGE.c:346
 54e:	2107      	movs	r1, #7
 550:	f105 0208 	add.w	r2, r5, #8	; 0x8
 554:	4643      	mov	r3, r8
 556:	f7ff fffe 	bl	0 <Show>
C:\Documents and Settings\jarek\Pulpit\Privet\Magisterka\Programy\1\um0427\FWLib\project/MESSAGE.c:347
 55a:	2009      	movs	r0, #9
 55c:	210a      	movs	r1, #10
 55e:	4a32      	ldr	r2, [pc, #200]	(628 <Show+0x628>)
 560:	4643      	mov	r3, r8
 562:	f7ff fffe 	bl	0 <Show>
C:\Documents and Settings\jarek\Pulpit\Privet\Magisterka\Programy\1\um0427\FWLib\project/MESSAGE.c:348
 566:	4633      	mov	r3, r6
 568:	2017      	movs	r0, #23
 56a:	210a      	movs	r1, #10
 56c:	4a2f      	ldr	r2, [pc, #188]	(62c <Show+0x62c>)
 56e:	f7ff fffe 	bl	0 <Show>
C:\Documents and Settings\jarek\Pulpit\Privet\Magisterka\Programy\1\um0427\FWLib\project/MESSAGE.c:349
 572:	230c      	movs	r3, #12
 574:	e1dd      	b.n	932 <Show+0x932>
C:\Documents and Settings\jarek\Pulpit\Privet\Magisterka\Programy\1\um0427\FWLib\project/MESSAGE.c:352
 576:	f7ff fffe 	bl	0 <KEY_CheckKey>
 57a:	2804      	cmp	r0, #4
 57c:	d00e      	beq.n	59c <Show+0x59c>
 57e:	dc04      	bgt.n	58a <Show+0x58a>
 580:	2801      	cmp	r0, #1
 582:	d00d      	beq.n	5a0 <Show+0x5a0>
 584:	2802      	cmp	r0, #2
 586:	d007      	beq.n	598 <Show+0x598>
 588:	e32c      	b.n	be4 <Show+0xbe4>
 58a:	f5b0 7f80 	cmp.w	r0, #256	; 0x100
 58e:	d04f      	beq.n	630 <Show+0x630>
 590:	f5b0 5f80 	cmp.w	r0, #4096	; 0x1000
 594:	d006      	beq.n	5a4 <Show+0x5a4>
 596:	e325      	b.n	be4 <Show+0xbe4>
C:\Documents and Settings\jarek\Pulpit\Privet\Magisterka\Programy\1\um0427\FWLib\project/MESSAGE.c:354
 598:	220e      	movs	r2, #14
 59a:	e1e2      	b.n	962 <Show+0x962>
C:\Documents and Settings\jarek\Pulpit\Privet\Magisterka\Programy\1\um0427\FWLib\project/MESSAGE.c:358
 59c:	220d      	movs	r2, #13
 59e:	e1e0      	b.n	962 <Show+0x962>
C:\Documents and Settings\jarek\Pulpit\Privet\Magisterka\Programy\1\um0427\FWLib\project/MESSAGE.c:362
 5a0:	220f      	movs	r2, #15
 5a2:	e1de      	b.n	962 <Show+0x962>
C:\Documents and Settings\jarek\Pulpit\Privet\Magisterka\Programy\1\um0427\FWLib\project/MESSAGE.c:366
 5a4:	4b1d      	ldr	r3, [pc, #116]	(61c <Show+0x61c>)
 5a6:	f893 3075 	ldrb.w	r3, [r3, #117]
 5aa:	2b05      	cmp	r3, #5
 5ac:	d004      	beq.n	5b8 <Show+0x5b8>
 5ae:	2b06      	cmp	r3, #6
 5b0:	d022      	beq.n	5f8 <Show+0x5f8>
 5b2:	2b04      	cmp	r3, #4
 5b4:	d011      	beq.n	5da <Show+0x5da>
 5b6:	e212      	b.n	9de <Show+0x9de>
C:\Documents and Settings\jarek\Pulpit\Privet\Magisterka\Programy\1\um0427\FWLib\project/MESSAGE.c:368
 5b8:	4c1a      	ldr	r4, [pc, #104]	(624 <Show+0x624>)
 5ba:	f44f 6261 	mov.w	r2, #3600	; 0xe10
 5be:	68a0      	ldr	r0, [r4, #8]
 5c0:	fbb0 f3f2 	udiv	r3, r0, r2
 5c4:	fb03 0212 	mls	r2, r3, r2, r0
 5c8:	233c      	movs	r3, #60
 5ca:	fbb2 f1f3 	udiv	r1, r2, r3
 5ce:	fb01 2313 	mls	r3, r1, r3, r2
 5d2:	2b3a      	cmp	r3, #58
 5d4:	d849      	bhi.n	66a <Show+0x66a>
C:\Documents and Settings\jarek\Pulpit\Privet\Magisterka\Programy\1\um0427\FWLib\project/MESSAGE.c:369
 5d6:	1c43      	adds	r3, r0, #1
 5d8:	e046      	b.n	668 <Show+0x668>
C:\Documents and Settings\jarek\Pulpit\Privet\Magisterka\Programy\1\um0427\FWLib\project/MESSAGE.c:374
 5da:	4c12      	ldr	r4, [pc, #72]	(624 <Show+0x624>)
 5dc:	f44f 6361 	mov.w	r3, #3600	; 0xe10
 5e0:	68a1      	ldr	r1, [r4, #8]
 5e2:	fbb1 f2f3 	udiv	r2, r1, r3
 5e6:	fb02 1313 	mls	r3, r2, r3, r1
 5ea:	f640 52d3 	movw	r2, #3539	; 0xdd3
 5ee:	4293      	cmp	r3, r2
 5f0:	d83b      	bhi.n	66a <Show+0x66a>
C:\Documents and Settings\jarek\Pulpit\Privet\Magisterka\Programy\1\um0427\FWLib\project/MESSAGE.c:375
 5f2:	f101 033c 	add.w	r3, r1, #60	; 0x3c
 5f6:	e037      	b.n	668 <Show+0x668>
C:\Documents and Settings\jarek\Pulpit\Privet\Magisterka\Programy\1\um0427\FWLib\project/MESSAGE.c:380
 5f8:	4c0a      	ldr	r4, [pc, #40]	(624 <Show+0x624>)
 5fa:	f44f 6361 	mov.w	r3, #3600	; 0xe10
 5fe:	68a0      	ldr	r0, [r4, #8]
 600:	2218      	movs	r2, #24
 602:	fbb0 f3f3 	udiv	r3, r0, r3
 606:	fbb3 f1f2 	udiv	r1, r3, r2
 60a:	fb01 3212 	mls	r2, r1, r2, r3
 60e:	2a16      	cmp	r2, #22
 610:	d82b      	bhi.n	66a <Show+0x66a>
C:\Documents and Settings\jarek\Pulpit\Privet\Magisterka\Programy\1\um0427\FWLib\project/MESSAGE.c:381
 612:	f500 6361 	add.w	r3, r0, #3600	; 0xe10
 616:	e027      	b.n	52 <Show+0x52>
 618:	00000028 	.word	0x00000028
 61c:	00000000 	.word	0x00000000
 620:	0000004d 	.word	0x0000004d
 624:	00000000 	.word	0x00000000
 628:	00000052 	.word	0x00000052
 62c:	0000005b 	.word	0x0000005b
C:\Documents and Settings\jarek\Pulpit\Privet\Magisterka\Programy\1\um0427\FWLib\project/MESSAGE.c:390
 630:	4ba9      	ldr	r3, [pc, #676]	(8d8 <Show+0x8d8>)
 632:	f893 3075 	ldrb.w	r3, [r3, #117]
 636:	2b05      	cmp	r3, #5
 638:	d004      	beq.n	644 <Show+0x644>
 63a:	2b06      	cmp	r3, #6
 63c:	d00d      	beq.n	65a <Show+0x65a>
 63e:	2b04      	cmp	r3, #4
 640:	d005      	beq.n	64e <Show+0x64e>
 642:	e1cc      	b.n	9de <Show+0x9de>
C:\Documents and Settings\jarek\Pulpit\Privet\Magisterka\Programy\1\um0427\FWLib\project/MESSAGE.c:392
 644:	4ca5      	ldr	r4, [pc, #660]	(8dc <Show+0x8dc>)
 646:	68a3      	ldr	r3, [r4, #8]
 648:	b17b      	cbz	r3, 66a <Show+0x66a>
C:\Documents and Settings\jarek\Pulpit\Privet\Magisterka\Programy\1\um0427\FWLib\project/MESSAGE.c:393
 64a:	3b01      	subs	r3, #1
 64c:	e00c      	b.n	668 <Show+0x668>
C:\Documents and Settings\jarek\Pulpit\Privet\Magisterka\Programy\1\um0427\FWLib\project/MESSAGE.c:398
 64e:	4ca3      	ldr	r4, [pc, #652]	(8dc <Show+0x8dc>)
 650:	68a3      	ldr	r3, [r4, #8]
 652:	2b3b      	cmp	r3, #59
 654:	d909      	bls.n	66a <Show+0x66a>
C:\Documents and Settings\jarek\Pulpit\Privet\Magisterka\Programy\1\um0427\FWLib\project/MESSAGE.c:399
 656:	3b3c      	subs	r3, #60
 658:	e006      	b.n	668 <Show+0x668>
C:\Documents and Settings\jarek\Pulpit\Privet\Magisterka\Programy\1\um0427\FWLib\project/MESSAGE.c:404
 65a:	4ca0      	ldr	r4, [pc, #640]	(8dc <Show+0x8dc>)
 65c:	68a3      	ldr	r3, [r4, #8]
 65e:	f5b3 6f61 	cmp.w	r3, #3600	; 0xe10
 662:	d302      	bcc.n	66a <Show+0x66a>
C:\Documents and Settings\jarek\Pulpit\Privet\Magisterka\Programy\1\um0427\FWLib\project/MESSAGE.c:405
 664:	f5a3 6361 	sub.w	r3, r3, #3600	; 0xe10
 668:	60a3      	str	r3, [r4, #8]
C:\Documents and Settings\jarek\Pulpit\Privet\Magisterka\Programy\1\um0427\FWLib\project/MESSAGE.c:407
 66a:	2009      	movs	r0, #9
 66c:	2107      	movs	r1, #7
 66e:	f104 0208 	add.w	r2, r4, #8	; 0x8
 672:	f994 300c 	ldrsb.w	r3, [r4, #12]
 676:	f7ff fffe 	bl	0 <Show>
 67a:	e1b0      	b.n	9de <Show+0x9de>
C:\Documents and Settings\jarek\Pulpit\Privet\Magisterka\Programy\1\um0427\FWLib\project/MESSAGE.c:415
 67c:	4b96      	ldr	r3, [pc, #600]	(8d8 <Show+0x8d8>)
 67e:	4d97      	ldr	r5, [pc, #604]	(8dc <Show+0x8dc>)
 680:	f893 3075 	ldrb.w	r3, [r3, #117]
 684:	3b02      	subs	r3, #2
 686:	2b04      	cmp	r3, #4
 688:	f200 8091 	bhi.w	7ae <Show+0x7ae>
 68c:	e8df f003 	tbb	[pc, r3]
 690:	03191903 	.word	0x03191903
 694:	0037      	.short	0x0037
C:\Documents and Settings\jarek\Pulpit\Privet\Magisterka\Programy\1\um0427\FWLib\project/MESSAGE.c:431
 696:	4a90      	ldr	r2, [pc, #576]	(8d8 <Show+0x8d8>)
C:\Documents and Settings\jarek\Pulpit\Privet\Magisterka\Programy\1\um0427\FWLib\project/MESSAGE.c:432
 698:	2400      	movs	r4, #0
C:\Documents and Settings\jarek\Pulpit\Privet\Magisterka\Programy\1\um0427\FWLib\project/MESSAGE.c:431
 69a:	2303      	movs	r3, #3
 69c:	f882 3075 	strb.w	r3, [r2, #117]
C:\Documents and Settings\jarek\Pulpit\Privet\Magisterka\Programy\1\um0427\FWLib\project/MESSAGE.c:433
 6a0:	2009      	movs	r0, #9
 6a2:	2107      	movs	r1, #7
 6a4:	4a8e      	ldr	r2, [pc, #568]	(8e0 <Show+0x8e0>)
 6a6:	4623      	mov	r3, r4
C:\Documents and Settings\jarek\Pulpit\Privet\Magisterka\Programy\1\um0427\FWLib\project/MESSAGE.c:432
 6a8:	60ec      	str	r4, [r5, #12]
C:\Documents and Settings\jarek\Pulpit\Privet\Magisterka\Programy\1\um0427\FWLib\project/MESSAGE.c:433
 6aa:	f7ff fffe 	bl	0 <Show>
C:\Documents and Settings\jarek\Pulpit\Privet\Magisterka\Programy\1\um0427\FWLib\project/MESSAGE.c:434
 6ae:	2009      	movs	r0, #9
 6b0:	210a      	movs	r1, #10
 6b2:	4a8c      	ldr	r2, [pc, #560]	(8e4 <Show+0x8e4>)
 6b4:	4623      	mov	r3, r4
 6b6:	f7ff fffe 	bl	0 <Show>
C:\Documents and Settings\jarek\Pulpit\Privet\Magisterka\Programy\1\um0427\FWLib\project/MESSAGE.c:435
 6ba:	2017      	movs	r0, #23
 6bc:	210a      	movs	r1, #10
 6be:	4a8a      	ldr	r2, [pc, #552]	(8e8 <Show+0x8e8>)
 6c0:	e052      	b.n	768 <Show+0x768>
C:\Documents and Settings\jarek\Pulpit\Privet\Magisterka\Programy\1\um0427\FWLib\project/MESSAGE.c:438
 6c2:	4a85      	ldr	r2, [pc, #532]	(8d8 <Show+0x8d8>)
 6c4:	2305      	movs	r3, #5
 6c6:	f882 3075 	strb.w	r3, [r2, #117]
C:\Documents and Settings\jarek\Pulpit\Privet\Magisterka\Programy\1\um0427\FWLib\project/MESSAGE.c:439
 6ca:	2301      	movs	r3, #1
 6cc:	60eb      	str	r3, [r5, #12]
C:\Documents and Settings\jarek\Pulpit\Privet\Magisterka\Programy\1\um0427\FWLib\project/MESSAGE.c:440
 6ce:	2009      	movs	r0, #9
 6d0:	210a      	movs	r1, #10
 6d2:	4a84      	ldr	r2, [pc, #528]	(8e4 <Show+0x8e4>)
 6d4:	3b01      	subs	r3, #1
 6d6:	e01c      	b.n	712 <Show+0x712>
C:\Documents and Settings\jarek\Pulpit\Privet\Magisterka\Programy\1\um0427\FWLib\project/MESSAGE.c:456
 6d8:	4b7f      	ldr	r3, [pc, #508]	(8d8 <Show+0x8d8>)
 6da:	4d80      	ldr	r5, [pc, #512]	(8dc <Show+0x8dc>)
 6dc:	f893 3075 	ldrb.w	r3, [r3, #117]
 6e0:	3b02      	subs	r3, #2
 6e2:	2b04      	cmp	r3, #4
 6e4:	d863      	bhi.n	7ae <Show+0x7ae>
 6e6:	e8df f003 	tbb	[pc, r3]
 6ea:	0324      	.short	0x0324
 6ec:	002a0a24 	.word	0x002a0a24
C:\Documents and Settings\jarek\Pulpit\Privet\Magisterka\Programy\1\um0427\FWLib\project/MESSAGE.c:465
 6f0:	4a79      	ldr	r2, [pc, #484]	(8d8 <Show+0x8d8>)
 6f2:	2302      	movs	r3, #2
C:\Documents and Settings\jarek\Pulpit\Privet\Magisterka\Programy\1\um0427\FWLib\project/MESSAGE.c:466
 6f4:	2400      	movs	r4, #0
C:\Documents and Settings\jarek\Pulpit\Privet\Magisterka\Programy\1\um0427\FWLib\project/MESSAGE.c:465
 6f6:	f882 3075 	strb.w	r3, [r2, #117]
C:\Documents and Settings\jarek\Pulpit\Privet\Magisterka\Programy\1\um0427\FWLib\project/MESSAGE.c:466
 6fa:	60ec      	str	r4, [r5, #12]
 6fc:	e025      	b.n	74a <Show+0x74a>
C:\Documents and Settings\jarek\Pulpit\Privet\Magisterka\Programy\1\um0427\FWLib\project/MESSAGE.c:472
 6fe:	4a76      	ldr	r2, [pc, #472]	(8d8 <Show+0x8d8>)
 700:	2304      	movs	r3, #4
 702:	f882 3075 	strb.w	r3, [r2, #117]
C:\Documents and Settings\jarek\Pulpit\Privet\Magisterka\Programy\1\um0427\FWLib\project/MESSAGE.c:473
 706:	2302      	movs	r3, #2
C:\Documents and Settings\jarek\Pulpit\Privet\Magisterka\Programy\1\um0427\FWLib\project/MESSAGE.c:474
 708:	4a76      	ldr	r2, [pc, #472]	(8e4 <Show+0x8e4>)
C:\Documents and Settings\jarek\Pulpit\Privet\Magisterka\Programy\1\um0427\FWLib\project/MESSAGE.c:473
 70a:	60eb      	str	r3, [r5, #12]
C:\Documents and Settings\jarek\Pulpit\Privet\Magisterka\Programy\1\um0427\FWLib\project/MESSAGE.c:474
 70c:	2009      	movs	r0, #9
 70e:	210a      	movs	r1, #10
 710:	2300      	movs	r3, #0
 712:	f7ff fffe 	bl	0 <Show>
C:\Documents and Settings\jarek\Pulpit\Privet\Magisterka\Programy\1\um0427\FWLib\project/MESSAGE.c:475
 716:	2017      	movs	r0, #23
 718:	210a      	movs	r1, #10
 71a:	2300      	movs	r3, #0
 71c:	4a72      	ldr	r2, [pc, #456]	(8e8 <Show+0x8e8>)
 71e:	f7ff fffe 	bl	0 <Show>
C:\Documents and Settings\jarek\Pulpit\Privet\Magisterka\Programy\1\um0427\FWLib\project/MESSAGE.c:476
 722:	2009      	movs	r0, #9
 724:	2107      	movs	r1, #7
 726:	4a6e      	ldr	r2, [pc, #440]	(8e0 <Show+0x8e0>)
 728:	f995 300c 	ldrsb.w	r3, [r5, #12]
 72c:	f7ff fffe 	bl	0 <Show>
C:\Documents and Settings\jarek\Pulpit\Privet\Magisterka\Programy\1\um0427\FWLib\project/MESSAGE.c:477
 730:	e03d      	b.n	7ae <Show+0x7ae>
C:\Documents and Settings\jarek\Pulpit\Privet\Magisterka\Programy\1\um0427\FWLib\project/MESSAGE.c:479
 732:	4a69      	ldr	r2, [pc, #420]	(8d8 <Show+0x8d8>)
 734:	2306      	movs	r3, #6
 736:	f882 3075 	strb.w	r3, [r2, #117]
C:\Documents and Settings\jarek\Pulpit\Privet\Magisterka\Programy\1\um0427\FWLib\project/MESSAGE.c:480
 73a:	2304      	movs	r3, #4
 73c:	e7e4      	b.n	708 <Show+0x708>
C:\Documents and Settings\jarek\Pulpit\Privet\Magisterka\Programy\1\um0427\FWLib\project/MESSAGE.c:487
 73e:	4b66      	ldr	r3, [pc, #408]	(8d8 <Show+0x8d8>)
C:\Documents and Settings\jarek\Pulpit\Privet\Magisterka\Programy\1\um0427\FWLib\project/MESSAGE.c:486
 740:	2400      	movs	r4, #0
C:\Documents and Settings\jarek\Pulpit\Privet\Magisterka\Programy\1\um0427\FWLib\project/MESSAGE.c:487
 742:	2202      	movs	r2, #2
C:\Documents and Settings\jarek\Pulpit\Privet\Magisterka\Programy\1\um0427\FWLib\project/MESSAGE.c:486
 744:	60ec      	str	r4, [r5, #12]
C:\Documents and Settings\jarek\Pulpit\Privet\Magisterka\Programy\1\um0427\FWLib\project/MESSAGE.c:487
 746:	f883 2075 	strb.w	r2, [r3, #117]
C:\Documents and Settings\jarek\Pulpit\Privet\Magisterka\Programy\1\um0427\FWLib\project/MESSAGE.c:488
 74a:	2009      	movs	r0, #9
 74c:	2107      	movs	r1, #7
 74e:	4a64      	ldr	r2, [pc, #400]	(8e0 <Show+0x8e0>)
 750:	4623      	mov	r3, r4
 752:	f7ff fffe 	bl	0 <Show>
C:\Documents and Settings\jarek\Pulpit\Privet\Magisterka\Programy\1\um0427\FWLib\project/MESSAGE.c:489
 756:	2017      	movs	r0, #23
 758:	210a      	movs	r1, #10
 75a:	4a63      	ldr	r2, [pc, #396]	(8e8 <Show+0x8e8>)
 75c:	4623      	mov	r3, r4
 75e:	f7ff fffe 	bl	0 <Show>
C:\Documents and Settings\jarek\Pulpit\Privet\Magisterka\Programy\1\um0427\FWLib\project/MESSAGE.c:490
 762:	4a60      	ldr	r2, [pc, #384]	(8e4 <Show+0x8e4>)
 764:	2009      	movs	r0, #9
 766:	210a      	movs	r1, #10
 768:	2301      	movs	r3, #1
 76a:	f7ff fffe 	bl	0 <Show>
 76e:	e01e      	b.n	7ae <Show+0x7ae>
C:\Documents and Settings\jarek\Pulpit\Privet\Magisterka\Programy\1\um0427\FWLib\project/MESSAGE.c:496
 770:	4b59      	ldr	r3, [pc, #356]	(8d8 <Show+0x8d8>)
 772:	f893 3075 	ldrb.w	r3, [r3, #117]
 776:	3b02      	subs	r3, #2
 778:	2b04      	cmp	r3, #4
 77a:	f200 8233 	bhi.w	be4 <Show+0xbe4>
 77e:	e8df f003 	tbb	[pc, r3]
 782:	1003      	.short	0x1003
 784:	00161616 	.word	0x00161616
C:\Documents and Settings\jarek\Pulpit\Privet\Magisterka\Programy\1\um0427\FWLib\project/MESSAGE.c:498
 788:	4c53      	ldr	r4, [pc, #332]	(8d8 <Show+0x8d8>)
 78a:	69a2      	ldr	r2, [r4, #24]
 78c:	6a23      	ldr	r3, [r4, #32]
 78e:	6013      	str	r3, [r2, #0]
C:\Documents and Settings\jarek\Pulpit\Privet\Magisterka\Programy\1\um0427\FWLib\project/MESSAGE.c:499
 790:	6b23      	ldr	r3, [r4, #48]
 792:	4798      	blx	r3
C:\Documents and Settings\jarek\Pulpit\Privet\Magisterka\Programy\1\um0427\FWLib\project/MESSAGE.c:500
 794:	4a51      	ldr	r2, [pc, #324]	(8dc <Show+0x8dc>)
 796:	6aa1      	ldr	r1, [r4, #40]
 798:	6893      	ldr	r3, [r2, #8]
 79a:	600b      	str	r3, [r1, #0]
C:\Documents and Settings\jarek\Pulpit\Privet\Magisterka\Programy\1\um0427\FWLib\project/MESSAGE.c:501
 79c:	2300      	movs	r3, #0
 79e:	7013      	strb	r3, [r2, #0]
C:\Documents and Settings\jarek\Pulpit\Privet\Magisterka\Programy\1\um0427\FWLib\project/MESSAGE.c:502
 7a0:	e220      	b.n	be4 <Show+0xbe4>
C:\Documents and Settings\jarek\Pulpit\Privet\Magisterka\Programy\1\um0427\FWLib\project/MESSAGE.c:504
 7a2:	4b4d      	ldr	r3, [pc, #308]	(8d8 <Show+0x8d8>)
 7a4:	6999      	ldr	r1, [r3, #24]
 7a6:	69da      	ldr	r2, [r3, #28]
C:\Documents and Settings\jarek\Pulpit\Privet\Magisterka\Programy\1\um0427\FWLib\project/MESSAGE.c:505
 7a8:	6b5b      	ldr	r3, [r3, #52]
C:\Documents and Settings\jarek\Pulpit\Privet\Magisterka\Programy\1\um0427\FWLib\project/MESSAGE.c:504
 7aa:	600a      	str	r2, [r1, #0]
 7ac:	e20f      	b.n	bce <Show+0xbce>
C:\Documents and Settings\jarek\Pulpit\Privet\Magisterka\Programy\1\um0427\FWLib\project/MESSAGE.c:515
 7ae:	220c      	movs	r2, #12
 7b0:	e216      	b.n	be0 <Show+0xbe0>
C:\Documents and Settings\jarek\Pulpit\Privet\Magisterka\Programy\1\um0427\FWLib\project/MESSAGE.c:522
 7b2:	f7ff fffe 	bl	0 <GRAPH_WhiteBlack>
C:\Documents and Settings\jarek\Pulpit\Privet\Magisterka\Programy\1\um0427\FWLib\project/MESSAGE.c:523
 7b6:	2103      	movs	r1, #3
 7b8:	2006      	movs	r0, #6
 7ba:	f7ff fffe 	bl	0 <GRAPH_TextGoTo>
C:\Documents and Settings\jarek\Pulpit\Privet\Magisterka\Programy\1\um0427\FWLib\project/MESSAGE.c:524
 7be:	484b      	ldr	r0, [pc, #300]	(130 <printf+0x130>)
 7c0:	f7ff fffe 	bl	0 <printf>
C:\Documents and Settings\jarek\Pulpit\Privet\Magisterka\Programy\1\um0427\FWLib\project/MESSAGE.c:525
 7c4:	2104      	movs	r1, #4
 7c6:	2006      	movs	r0, #6
 7c8:	f7ff fffe 	bl	0 <GRAPH_TextGoTo>
C:\Documents and Settings\jarek\Pulpit\Privet\Magisterka\Programy\1\um0427\FWLib\project/MESSAGE.c:526
 7cc:	4847      	ldr	r0, [pc, #284]	(120 <printf+0x120>)
 7ce:	f7ff fffe 	bl	0 <printf>
C:\Documents and Settings\jarek\Pulpit\Privet\Magisterka\Programy\1\um0427\FWLib\project/MESSAGE.c:527
 7d2:	2105      	movs	r1, #5
 7d4:	2006      	movs	r0, #6
 7d6:	f7ff fffe 	bl	0 <GRAPH_TextGoTo>
C:\Documents and Settings\jarek\Pulpit\Privet\Magisterka\Programy\1\um0427\FWLib\project/MESSAGE.c:528
 7da:	4844      	ldr	r0, [pc, #272]	(114 <printf+0x114>)
 7dc:	f7ff fffe 	bl	0 <printf>
C:\Documents and Settings\jarek\Pulpit\Privet\Magisterka\Programy\1\um0427\FWLib\project/MESSAGE.c:529
 7e0:	2006      	movs	r0, #6
 7e2:	4601      	mov	r1, r0
 7e4:	f7ff fffe 	bl	0 <GRAPH_TextGoTo>
C:\Documents and Settings\jarek\Pulpit\Privet\Magisterka\Programy\1\um0427\FWLib\project/MESSAGE.c:530
 7e8:	4840      	ldr	r0, [pc, #256]	(104 <printf+0x104>)
 7ea:	f7ff fffe 	bl	0 <printf>
C:\Documents and Settings\jarek\Pulpit\Privet\Magisterka\Programy\1\um0427\FWLib\project/MESSAGE.c:531
 7ee:	2107      	movs	r1, #7
 7f0:	2006      	movs	r0, #6
 7f2:	f7ff fffe 	bl	0 <GRAPH_TextGoTo>
C:\Documents and Settings\jarek\Pulpit\Privet\Magisterka\Programy\1\um0427\FWLib\project/MESSAGE.c:532
 7f6:	483d      	ldr	r0, [pc, #244]	(f8 <printf+0xf8>)
 7f8:	f7ff fffe 	bl	0 <printf>
C:\Documents and Settings\jarek\Pulpit\Privet\Magisterka\Programy\1\um0427\FWLib\project/MESSAGE.c:533
 7fc:	2108      	movs	r1, #8
 7fe:	2006      	movs	r0, #6
 800:	f7ff fffe 	bl	0 <GRAPH_TextGoTo>
C:\Documents and Settings\jarek\Pulpit\Privet\Magisterka\Programy\1\um0427\FWLib\project/MESSAGE.c:534
 804:	4839      	ldr	r0, [pc, #228]	(e8 <printf+0xe8>)
 806:	f7ff fffe 	bl	0 <printf>
C:\Documents and Settings\jarek\Pulpit\Privet\Magisterka\Programy\1\um0427\FWLib\project/MESSAGE.c:535
 80a:	2109      	movs	r1, #9
 80c:	2006      	movs	r0, #6
 80e:	f7ff fffe 	bl	0 <GRAPH_TextGoTo>
C:\Documents and Settings\jarek\Pulpit\Privet\Magisterka\Programy\1\um0427\FWLib\project/MESSAGE.c:536
 812:	4836      	ldr	r0, [pc, #216]	(dc <printf+0xdc>)
 814:	f7ff fffe 	bl	0 <printf>
C:\Documents and Settings\jarek\Pulpit\Privet\Magisterka\Programy\1\um0427\FWLib\project/MESSAGE.c:537
 818:	210a      	movs	r1, #10
 81a:	2006      	movs	r0, #6
 81c:	f7ff fffe 	bl	0 <GRAPH_TextGoTo>
C:\Documents and Settings\jarek\Pulpit\Privet\Magisterka\Programy\1\um0427\FWLib\project/MESSAGE.c:538
 820:	4832      	ldr	r0, [pc, #200]	(cc <printf+0xcc>)
 822:	f7ff fffe 	bl	0 <printf>
C:\Documents and Settings\jarek\Pulpit\Privet\Magisterka\Programy\1\um0427\FWLib\project/MESSAGE.c:540
 826:	2500      	movs	r5, #0
 828:	2024      	movs	r0, #36
 82a:	210f      	movs	r1, #15
 82c:	22a8      	movs	r2, #168
 82e:	234e      	movs	r3, #78
C:\Documents and Settings\jarek\Pulpit\Privet\Magisterka\Programy\1\um0427\FWLib\project/MESSAGE.c:541
 830:	2401      	movs	r4, #1
C:\Documents and Settings\jarek\Pulpit\Privet\Magisterka\Programy\1\um0427\FWLib\project/MESSAGE.c:540
 832:	9500      	str	r5, [sp, #0]
 834:	f7ff fffe 	bl	0 <GRAPH_RectangleFilled>
C:\Documents and Settings\jarek\Pulpit\Privet\Magisterka\Programy\1\um0427\FWLib\project/MESSAGE.c:541
 838:	210f      	movs	r1, #15
 83a:	22a8      	movs	r2, #168
 83c:	234e      	movs	r3, #78
 83e:	2024      	movs	r0, #36
 840:	9400      	str	r4, [sp, #0]
 842:	f7ff fffe 	bl	0 <GRAPH_Rectangle>
C:\Documents and Settings\jarek\Pulpit\Privet\Magisterka\Programy\1\um0427\FWLib\project/MESSAGE.c:542
 846:	20cc      	movs	r0, #204
 848:	2110      	movs	r1, #16
 84a:	235d      	movs	r3, #93
 84c:	4602      	mov	r2, r0
 84e:	9400      	str	r4, [sp, #0]
 850:	f7ff fffe 	bl	0 <GRAPH_Line>
C:\Documents and Settings\jarek\Pulpit\Privet\Magisterka\Programy\1\um0427\FWLib\project/MESSAGE.c:543
 854:	215d      	movs	r1, #93
 856:	460b      	mov	r3, r1
 858:	22cc      	movs	r2, #204
 85a:	9400      	str	r4, [sp, #0]
 85c:	2025      	movs	r0, #37
C:\Documents and Settings\jarek\Pulpit\Privet\Magisterka\Programy\1\um0427\FWLib\project/MESSAGE.c:546
 85e:	4c1e      	ldr	r4, [pc, #120]	(8d8 <Show+0x8d8>)
C:\Documents and Settings\jarek\Pulpit\Privet\Magisterka\Programy\1\um0427\FWLib\project/MESSAGE.c:543
 860:	f7ff fffe 	bl	0 <GRAPH_Line>
C:\Documents and Settings\jarek\Pulpit\Privet\Magisterka\Programy\1\um0427\FWLib\project/MESSAGE.c:545
 864:	2103      	movs	r1, #3
 866:	2007      	movs	r0, #7
 868:	f7ff fffe 	bl	0 <GRAPH_TextGoTo>
C:\Documents and Settings\jarek\Pulpit\Privet\Magisterka\Programy\1\um0427\FWLib\project/MESSAGE.c:546
 86c:	6820      	ldr	r0, [r4, #0]
 86e:	f7ff fffe 	bl	0 <printf>
C:\Documents and Settings\jarek\Pulpit\Privet\Magisterka\Programy\1\um0427\FWLib\project/MESSAGE.c:548
 872:	2104      	movs	r1, #4
 874:	2007      	movs	r0, #7
 876:	f7ff fffe 	bl	0 <GRAPH_TextGoTo>
C:\Documents and Settings\jarek\Pulpit\Privet\Magisterka\Programy\1\um0427\FWLib\project/MESSAGE.c:549
 87a:	6860      	ldr	r0, [r4, #4]
 87c:	f7ff fffe 	bl	0 <printf>
C:\Documents and Settings\jarek\Pulpit\Privet\Magisterka\Programy\1\um0427\FWLib\project/MESSAGE.c:551
 880:	2105      	movs	r1, #5
 882:	2007      	movs	r0, #7
 884:	f7ff fffe 	bl	0 <GRAPH_TextGoTo>
C:\Documents and Settings\jarek\Pulpit\Privet\Magisterka\Programy\1\um0427\FWLib\project/MESSAGE.c:552
 888:	68a0      	ldr	r0, [r4, #8]
 88a:	f7ff fffe 	bl	0 <printf>
C:\Documents and Settings\jarek\Pulpit\Privet\Magisterka\Programy\1\um0427\FWLib\project/MESSAGE.c:554
 88e:	2106      	movs	r1, #6
 890:	2007      	movs	r0, #7
 892:	f7ff fffe 	bl	0 <GRAPH_TextGoTo>
C:\Documents and Settings\jarek\Pulpit\Privet\Magisterka\Programy\1\um0427\FWLib\project/MESSAGE.c:555
 896:	68e0      	ldr	r0, [r4, #12]
 898:	f7ff fffe 	bl	0 <printf>
C:\Documents and Settings\jarek\Pulpit\Privet\Magisterka\Programy\1\um0427\FWLib\project/MESSAGE.c:557
 89c:	2007      	movs	r0, #7
 89e:	4601      	mov	r1, r0
 8a0:	f7ff fffe 	bl	0 <GRAPH_TextGoTo>
C:\Documents and Settings\jarek\Pulpit\Privet\Magisterka\Programy\1\um0427\FWLib\project/MESSAGE.c:558
 8a4:	6920      	ldr	r0, [r4, #16]
 8a6:	f7ff fffe 	bl	0 <printf>
C:\Documents and Settings\jarek\Pulpit\Privet\Magisterka\Programy\1\um0427\FWLib\project/MESSAGE.c:560
 8aa:	2108      	movs	r1, #8
 8ac:	2007      	movs	r0, #7
 8ae:	f7ff fffe 	bl	0 <GRAPH_TextGoTo>
C:\Documents and Settings\jarek\Pulpit\Privet\Magisterka\Programy\1\um0427\FWLib\project/MESSAGE.c:561
 8b2:	6960      	ldr	r0, [r4, #20]
 8b4:	f7ff fffe 	bl	0 <printf>
C:\Documents and Settings\jarek\Pulpit\Privet\Magisterka\Programy\1\um0427\FWLib\project/MESSAGE.c:563
 8b8:	2303      	movs	r3, #3
 8ba:	f884 3075 	strb.w	r3, [r4, #117]
C:\Documents and Settings\jarek\Pulpit\Privet\Magisterka\Programy\1\um0427\FWLib\project/MESSAGE.c:565
 8be:	2009      	movs	r0, #9
 8c0:	2107      	movs	r1, #7
 8c2:	f7ff fffe 	bl	0 <GRAPH_TextGoTo>
 8c6:	4628      	mov	r0, r5
C:\Documents and Settings\jarek\Pulpit\Privet\Magisterka\Programy\1\um0427\FWLib\project/MESSAGE.c:566
 8c8:	e01b      	b.n	902 <Show+0x902>
C:\Documents and Settings\jarek\Pulpit\Privet\Magisterka\Programy\1\um0427\FWLib\project/MESSAGE.c:567
 8ca:	6ad2      	ldr	r2, [r2, #44]
 8cc:	5683      	ldrsb	r3, [r0, r2]
 8ce:	b9bb      	cbnz	r3, 900 <Show+0x900>
C:\Documents and Settings\jarek\Pulpit\Privet\Magisterka\Programy\1\um0427\FWLib\project/MESSAGE.c:568
 8d0:	3320      	adds	r3, #32
 8d2:	5483      	strb	r3, [r0, r2]
 8d4:	4601      	mov	r1, r0
C:\Documents and Settings\jarek\Pulpit\Privet\Magisterka\Programy\1\um0427\FWLib\project/MESSAGE.c:569
 8d6:	e010      	b.n	8fa <Show+0x8fa>
	...
 8e0:	00000008 	.word	0x00000008
 8e4:	00000052 	.word	0x00000052
 8e8:	0000005b 	.word	0x0000005b
 8ec:	00000028 	.word	0x00000028
C:\Documents and Settings\jarek\Pulpit\Privet\Magisterka\Programy\1\um0427\FWLib\project/MESSAGE.c:570
 8f0:	4ba4      	ldr	r3, [pc, #656]	(b84 <Show+0xb84>)
 8f2:	6ada      	ldr	r2, [r3, #44]
 8f4:	2320      	movs	r3, #32
 8f6:	5453      	strb	r3, [r2, r1]
 8f8:	3101      	adds	r1, #1
C:\Documents and Settings\jarek\Pulpit\Privet\Magisterka\Programy\1\um0427\FWLib\project/MESSAGE.c:569
 8fa:	290a      	cmp	r1, #10
 8fc:	d1f8      	bne.n	8f0 <Show+0x8f0>
 8fe:	200a      	movs	r0, #10
C:\Documents and Settings\jarek\Pulpit\Privet\Magisterka\Programy\1\um0427\FWLib\project/MESSAGE.c:566
 900:	3001      	adds	r0, #1
 902:	2809      	cmp	r0, #9
 904:	4a9f      	ldr	r2, [pc, #636]	(b84 <Show+0xb84>)
 906:	dde0      	ble.n	8ca <Show+0x8ca>
C:\Documents and Settings\jarek\Pulpit\Privet\Magisterka\Programy\1\um0427\FWLib\project/MESSAGE.c:574
 908:	6ad3      	ldr	r3, [r2, #44]
C:\Documents and Settings\jarek\Pulpit\Privet\Magisterka\Programy\1\um0427\FWLib\project/MESSAGE.c:566
 90a:	4d9f      	ldr	r5, [pc, #636]	(b88 <Show+0xb88>)
C:\Documents and Settings\jarek\Pulpit\Privet\Magisterka\Programy\1\um0427\FWLib\project/MESSAGE.c:574
 90c:	2400      	movs	r4, #0
C:\Documents and Settings\jarek\Pulpit\Privet\Magisterka\Programy\1\um0427\FWLib\project/MESSAGE.c:566
 90e:	6068      	str	r0, [r5, #4]
C:\Documents and Settings\jarek\Pulpit\Privet\Magisterka\Programy\1\um0427\FWLib\project/MESSAGE.c:574
 910:	725c      	strb	r4, [r3, #9]
C:\Documents and Settings\jarek\Pulpit\Privet\Magisterka\Programy\1\um0427\FWLib\project/MESSAGE.c:575
 912:	6ad0      	ldr	r0, [r2, #44]
 914:	f7ff fffe 	bl	0 <printf>
C:\Documents and Settings\jarek\Pulpit\Privet\Magisterka\Programy\1\um0427\FWLib\project/MESSAGE.c:577
 918:	2009      	movs	r0, #9
 91a:	210a      	movs	r1, #10
 91c:	4a9b      	ldr	r2, [pc, #620]	(b8c <Show+0xb8c>)
 91e:	4623      	mov	r3, r4
 920:	f7ff fffe 	bl	0 <Show>
C:\Documents and Settings\jarek\Pulpit\Privet\Magisterka\Programy\1\um0427\FWLib\project/MESSAGE.c:578
 924:	2301      	movs	r3, #1
 926:	2017      	movs	r0, #23
 928:	210a      	movs	r1, #10
 92a:	4a99      	ldr	r2, [pc, #612]	(b90 <Show+0xb90>)
 92c:	f7ff fffe 	bl	0 <Show>
C:\Documents and Settings\jarek\Pulpit\Privet\Magisterka\Programy\1\um0427\FWLib\project/MESSAGE.c:579
 930:	2311      	movs	r3, #17
 932:	702b      	strb	r3, [r5, #0]
C:\Documents and Settings\jarek\Pulpit\Privet\Magisterka\Programy\1\um0427\FWLib\project/MESSAGE.c:580
 934:	e156      	b.n	be4 <Show+0xbe4>
C:\Documents and Settings\jarek\Pulpit\Privet\Magisterka\Programy\1\um0427\FWLib\project/MESSAGE.c:582
 936:	f7ff fffe 	bl	0 <KEY_CheckKey>
 93a:	2804      	cmp	r0, #4
 93c:	d00e      	beq.n	95c <Show+0x95c>
 93e:	dc04      	bgt.n	94a <Show+0x94a>
 940:	2801      	cmp	r0, #1
 942:	d00d      	beq.n	960 <Show+0x960>
 944:	2802      	cmp	r0, #2
 946:	d007      	beq.n	958 <Show+0x958>
 948:	e14c      	b.n	be4 <Show+0xbe4>
 94a:	f5b0 7f80 	cmp.w	r0, #256	; 0x100
 94e:	d029      	beq.n	9a4 <Show+0x9a4>
 950:	f5b0 5f80 	cmp.w	r0, #4096	; 0x1000
 954:	d008      	beq.n	968 <Show+0x968>
 956:	e145      	b.n	be4 <Show+0xbe4>
C:\Documents and Settings\jarek\Pulpit\Privet\Magisterka\Programy\1\um0427\FWLib\project/MESSAGE.c:584
 958:	2213      	movs	r2, #19
 95a:	e002      	b.n	962 <Show+0x962>
C:\Documents and Settings\jarek\Pulpit\Privet\Magisterka\Programy\1\um0427\FWLib\project/MESSAGE.c:588
 95c:	2212      	movs	r2, #18
 95e:	e000      	b.n	962 <Show+0x962>
C:\Documents and Settings\jarek\Pulpit\Privet\Magisterka\Programy\1\um0427\FWLib\project/MESSAGE.c:592
 960:	2214      	movs	r2, #20
 962:	4b89      	ldr	r3, [pc, #548]	(b88 <Show+0xb88>)
 964:	701a      	strb	r2, [r3, #0]
 966:	e03a      	b.n	9de <Show+0x9de>
C:\Documents and Settings\jarek\Pulpit\Privet\Magisterka\Programy\1\um0427\FWLib\project/MESSAGE.c:596
 968:	4b86      	ldr	r3, [pc, #536]	(b84 <Show+0xb84>)
 96a:	f893 3075 	ldrb.w	r3, [r3, #117]
 96e:	3b07      	subs	r3, #7
 970:	2b07      	cmp	r3, #7
 972:	d834      	bhi.n	9de <Show+0x9de>
 974:	e8df f003 	tbb	[pc, r3]
 978:	0a080604 	.word	0x0a080604
 97c:	12100e0c 	.word	0x12100e0c
C:\Documents and Settings\jarek\Pulpit\Privet\Magisterka\Programy\1\um0427\FWLib\project/MESSAGE.c:598
 980:	2001      	movs	r0, #1
 982:	e00c      	b.n	99e <Show+0x99e>
C:\Documents and Settings\jarek\Pulpit\Privet\Magisterka\Programy\1\um0427\FWLib\project/MESSAGE.c:601
 984:	2002      	movs	r0, #2
 986:	e00a      	b.n	99e <Show+0x99e>
C:\Documents and Settings\jarek\Pulpit\Privet\Magisterka\Programy\1\um0427\FWLib\project/MESSAGE.c:604
 988:	2003      	movs	r0, #3
 98a:	e008      	b.n	99e <Show+0x99e>
C:\Documents and Settings\jarek\Pulpit\Privet\Magisterka\Programy\1\um0427\FWLib\project/MESSAGE.c:607
 98c:	2004      	movs	r0, #4
 98e:	e006      	b.n	99e <Show+0x99e>
C:\Documents and Settings\jarek\Pulpit\Privet\Magisterka\Programy\1\um0427\FWLib\project/MESSAGE.c:610
 990:	2005      	movs	r0, #5
 992:	e004      	b.n	99e <Show+0x99e>
C:\Documents and Settings\jarek\Pulpit\Privet\Magisterka\Programy\1\um0427\FWLib\project/MESSAGE.c:613
 994:	2006      	movs	r0, #6
 996:	e002      	b.n	99e <Show+0x99e>
C:\Documents and Settings\jarek\Pulpit\Privet\Magisterka\Programy\1\um0427\FWLib\project/MESSAGE.c:616
 998:	2007      	movs	r0, #7
 99a:	e000      	b.n	99e <Show+0x99e>
C:\Documents and Settings\jarek\Pulpit\Privet\Magisterka\Programy\1\um0427\FWLib\project/MESSAGE.c:619
 99c:	2008      	movs	r0, #8
 99e:	f7ff fffe 	bl	0 <Show>
 9a2:	e01c      	b.n	9de <Show+0x9de>
C:\Documents and Settings\jarek\Pulpit\Privet\Magisterka\Programy\1\um0427\FWLib\project/MESSAGE.c:626
 9a4:	4b77      	ldr	r3, [pc, #476]	(b84 <Show+0xb84>)
 9a6:	f893 3075 	ldrb.w	r3, [r3, #117]
 9aa:	3b07      	subs	r3, #7
 9ac:	2b07      	cmp	r3, #7
 9ae:	d816      	bhi.n	9de <Show+0x9de>
 9b0:	e8df f003 	tbb	[pc, r3]
 9b4:	0a080604 	.word	0x0a080604
 9b8:	12100e0c 	.word	0x12100e0c
C:\Documents and Settings\jarek\Pulpit\Privet\Magisterka\Programy\1\um0427\FWLib\project/MESSAGE.c:628
 9bc:	2001      	movs	r0, #1
 9be:	e00c      	b.n	9da <Show+0x9da>
C:\Documents and Settings\jarek\Pulpit\Privet\Magisterka\Programy\1\um0427\FWLib\project/MESSAGE.c:631
 9c0:	2002      	movs	r0, #2
 9c2:	e00a      	b.n	9da <Show+0x9da>
C:\Documents and Settings\jarek\Pulpit\Privet\Magisterka\Programy\1\um0427\FWLib\project/MESSAGE.c:634
 9c4:	2003      	movs	r0, #3
 9c6:	e008      	b.n	9da <Show+0x9da>
C:\Documents and Settings\jarek\Pulpit\Privet\Magisterka\Programy\1\um0427\FWLib\project/MESSAGE.c:637
 9c8:	2004      	movs	r0, #4
 9ca:	e006      	b.n	9da <Show+0x9da>
C:\Documents and Settings\jarek\Pulpit\Privet\Magisterka\Programy\1\um0427\FWLib\project/MESSAGE.c:640
 9cc:	2005      	movs	r0, #5
 9ce:	e004      	b.n	9da <Show+0x9da>
C:\Documents and Settings\jarek\Pulpit\Privet\Magisterka\Programy\1\um0427\FWLib\project/MESSAGE.c:643
 9d0:	2006      	movs	r0, #6
 9d2:	e002      	b.n	9da <Show+0x9da>
C:\Documents and Settings\jarek\Pulpit\Privet\Magisterka\Programy\1\um0427\FWLib\project/MESSAGE.c:646
 9d4:	2007      	movs	r0, #7
 9d6:	e000      	b.n	9da <Show+0x9da>
C:\Documents and Settings\jarek\Pulpit\Privet\Magisterka\Programy\1\um0427\FWLib\project/MESSAGE.c:649
 9d8:	2008      	movs	r0, #8
 9da:	f7ff fffe 	bl	0 <Show>
C:\Documents and Settings\jarek\Pulpit\Privet\Magisterka\Programy\1\um0427\FWLib\project/MESSAGE.c:653
 9de:	f7ff fffe 	bl	0 <KEY_KeyServed>
 9e2:	e0ff      	b.n	be4 <Show+0xbe4>
C:\Documents and Settings\jarek\Pulpit\Privet\Magisterka\Programy\1\um0427\FWLib\project/MESSAGE.c:658
 9e4:	4b67      	ldr	r3, [pc, #412]	(b84 <Show+0xb84>)
 9e6:	f893 3075 	ldrb.w	r3, [r3, #117]
 9ea:	3b02      	subs	r3, #2
 9ec:	2b0c      	cmp	r3, #12
 9ee:	f200 80f6 	bhi.w	bde <Show+0xbde>
 9f2:	e8df f013 	tbh	[pc, r3, lsl #1]
 9f6:	000d      	.short	0x000d
 9f8:	00f40026 	.word	0x00f40026
 9fc:	00f400f4 	.word	0x00f400f4
 a00:	009200a3 	.word	0x009200a3
 a04:	006e0080 	.word	0x006e0080
 a08:	0048005c 	.word	0x0048005c
 a0c:	00120026 	.word	0x00120026
C:\Documents and Settings\jarek\Pulpit\Privet\Magisterka\Programy\1\um0427\FWLib\project/MESSAGE.c:660
 a10:	4b5c      	ldr	r3, [pc, #368]	(b84 <Show+0xb84>)
 a12:	2203      	movs	r2, #3
 a14:	f883 2075 	strb.w	r2, [r3, #117]
 a18:	e006      	b.n	a28 <Show+0xa28>
C:\Documents and Settings\jarek\Pulpit\Privet\Magisterka\Programy\1\um0427\FWLib\project/MESSAGE.c:671
 a1a:	4b5a      	ldr	r3, [pc, #360]	(b84 <Show+0xb84>)
 a1c:	2203      	movs	r2, #3
 a1e:	f883 2075 	strb.w	r2, [r3, #117]
C:\Documents and Settings\jarek\Pulpit\Privet\Magisterka\Programy\1\um0427\FWLib\project/MESSAGE.c:672
 a22:	2000      	movs	r0, #0
 a24:	f7ff fffe 	bl	0 <Show>
C:\Documents and Settings\jarek\Pulpit\Privet\Magisterka\Programy\1\um0427\FWLib\project/MESSAGE.c:673
 a28:	2009      	movs	r0, #9
 a2a:	210a      	movs	r1, #10
 a2c:	4a57      	ldr	r2, [pc, #348]	(b8c <Show+0xb8c>)
 a2e:	2300      	movs	r3, #0
 a30:	f7ff fffe 	bl	0 <Show>
C:\Documents and Settings\jarek\Pulpit\Privet\Magisterka\Programy\1\um0427\FWLib\project/MESSAGE.c:674
 a34:	4a56      	ldr	r2, [pc, #344]	(b90 <Show+0xb90>)
 a36:	2017      	movs	r0, #23
 a38:	210a      	movs	r1, #10
 a3a:	2301      	movs	r3, #1
 a3c:	f7ff fffe 	bl	0 <Show>
C:\Documents and Settings\jarek\Pulpit\Privet\Magisterka\Programy\1\um0427\FWLib\project/MESSAGE.c:675
 a40:	e0cd      	b.n	bde <Show+0xbde>
C:\Documents and Settings\jarek\Pulpit\Privet\Magisterka\Programy\1\um0427\FWLib\project/MESSAGE.c:677
 a42:	4b50      	ldr	r3, [pc, #320]	(b84 <Show+0xb84>)
 a44:	220e      	movs	r2, #14
 a46:	f883 2075 	strb.w	r2, [r3, #117]
C:\Documents and Settings\jarek\Pulpit\Privet\Magisterka\Programy\1\um0427\FWLib\project/MESSAGE.c:678
 a4a:	2009      	movs	r0, #9
 a4c:	210a      	movs	r1, #10
 a4e:	4a4f      	ldr	r2, [pc, #316]	(b8c <Show+0xb8c>)
 a50:	2300      	movs	r3, #0
 a52:	f7ff fffe 	bl	0 <Show>
C:\Documents and Settings\jarek\Pulpit\Privet\Magisterka\Programy\1\um0427\FWLib\project/MESSAGE.c:679
 a56:	2017      	movs	r0, #23
 a58:	210a      	movs	r1, #10
 a5a:	4a4d      	ldr	r2, [pc, #308]	(b90 <Show+0xb90>)
 a5c:	2300      	movs	r3, #0
 a5e:	f7ff fffe 	bl	0 <Show>
C:\Documents and Settings\jarek\Pulpit\Privet\Magisterka\Programy\1\um0427\FWLib\project/MESSAGE.c:680
 a62:	2008      	movs	r0, #8
 a64:	e020      	b.n	aa8 <Show+0xaa8>
C:\Documents and Settings\jarek\Pulpit\Privet\Magisterka\Programy\1\um0427\FWLib\project/MESSAGE.c:724
 a66:	4b47      	ldr	r3, [pc, #284]	(b84 <Show+0xb84>)
 a68:	f893 3075 	ldrb.w	r3, [r3, #117]
 a6c:	3b02      	subs	r3, #2
 a6e:	2b0c      	cmp	r3, #12
 a70:	f200 80b5 	bhi.w	bde <Show+0xbde>
 a74:	e8df f003 	tbb	[pc, r3]
 a78:	b3b38e74 	.word	0xb3b38e74
 a7c:	62748eb3 	.word	0x62748eb3
 a80:	1b2d3f51 	.word	0x1b2d3f51
 a84:	0007      	.short	0x0007
C:\Documents and Settings\jarek\Pulpit\Privet\Magisterka\Programy\1\um0427\FWLib\project/MESSAGE.c:738
 a86:	4b3f      	ldr	r3, [pc, #252]	(b84 <Show+0xb84>)
 a88:	220d      	movs	r2, #13
 a8a:	f883 2075 	strb.w	r2, [r3, #117]
C:\Documents and Settings\jarek\Pulpit\Privet\Magisterka\Programy\1\um0427\FWLib\project/MESSAGE.c:739
 a8e:	2009      	movs	r0, #9
 a90:	210a      	movs	r1, #10
 a92:	4a3e      	ldr	r2, [pc, #248]	(b8c <Show+0xb8c>)
 a94:	2300      	movs	r3, #0
 a96:	f7ff fffe 	bl	0 <Show>
C:\Documents and Settings\jarek\Pulpit\Privet\Magisterka\Programy\1\um0427\FWLib\project/MESSAGE.c:740
 a9a:	2017      	movs	r0, #23
 a9c:	210a      	movs	r1, #10
 a9e:	4a3c      	ldr	r2, [pc, #240]	(b90 <Show+0xb90>)
 aa0:	2300      	movs	r3, #0
 aa2:	f7ff fffe 	bl	0 <Show>
C:\Documents and Settings\jarek\Pulpit\Privet\Magisterka\Programy\1\um0427\FWLib\project/MESSAGE.c:741
 aa6:	2007      	movs	r0, #7
 aa8:	f7ff fffe 	bl	0 <Show>
C:\Documents and Settings\jarek\Pulpit\Privet\Magisterka\Programy\1\um0427\FWLib\project/MESSAGE.c:742
 aac:	e097      	b.n	bde <Show+0xbde>
C:\Documents and Settings\jarek\Pulpit\Privet\Magisterka\Programy\1\um0427\FWLib\project/MESSAGE.c:744
 aae:	4b35      	ldr	r3, [pc, #212]	(b84 <Show+0xb84>)
 ab0:	220c      	movs	r2, #12
 ab2:	f883 2075 	strb.w	r2, [r3, #117]
C:\Documents and Settings\jarek\Pulpit\Privet\Magisterka\Programy\1\um0427\FWLib\project/MESSAGE.c:745
 ab6:	2009      	movs	r0, #9
 ab8:	210a      	movs	r1, #10
 aba:	4a34      	ldr	r2, [pc, #208]	(b8c <Show+0xb8c>)
 abc:	2300      	movs	r3, #0
 abe:	f7ff fffe 	bl	0 <Show>
C:\Documents and Settings\jarek\Pulpit\Privet\Magisterka\Programy\1\um0427\FWLib\project/MESSAGE.c:746
 ac2:	2017      	movs	r0, #23
 ac4:	210a      	movs	r1, #10
 ac6:	4a32      	ldr	r2, [pc, #200]	(b90 <Show+0xb90>)
 ac8:	2300      	movs	r3, #0
 aca:	f7ff fffe 	bl	0 <Show>
C:\Documents and Settings\jarek\Pulpit\Privet\Magisterka\Programy\1\um0427\FWLib\project/MESSAGE.c:747
 ace:	2006      	movs	r0, #6
 ad0:	e7ea      	b.n	aa8 <Show+0xaa8>
C:\Documents and Settings\jarek\Pulpit\Privet\Magisterka\Programy\1\um0427\FWLib\project/MESSAGE.c:750
 ad2:	4b2c      	ldr	r3, [pc, #176]	(b84 <Show+0xb84>)
 ad4:	220b      	movs	r2, #11
 ad6:	f883 2075 	strb.w	r2, [r3, #117]
C:\Documents and Settings\jarek\Pulpit\Privet\Magisterka\Programy\1\um0427\FWLib\project/MESSAGE.c:751
 ada:	2009      	movs	r0, #9
 adc:	210a      	movs	r1, #10
 ade:	4a2b      	ldr	r2, [pc, #172]	(b8c <Show+0xb8c>)
 ae0:	2300      	movs	r3, #0
 ae2:	f7ff fffe 	bl	0 <Show>
C:\Documents and Settings\jarek\Pulpit\Privet\Magisterka\Programy\1\um0427\FWLib\project/MESSAGE.c:752
 ae6:	2017      	movs	r0, #23
 ae8:	210a      	movs	r1, #10
 aea:	4a29      	ldr	r2, [pc, #164]	(b90 <Show+0xb90>)
 aec:	2300      	movs	r3, #0
 aee:	f7ff fffe 	bl	0 <Show>
C:\Documents and Settings\jarek\Pulpit\Privet\Magisterka\Programy\1\um0427\FWLib\project/MESSAGE.c:753
 af2:	2005      	movs	r0, #5
 af4:	e7d8      	b.n	aa8 <Show+0xaa8>
C:\Documents and Settings\jarek\Pulpit\Privet\Magisterka\Programy\1\um0427\FWLib\project/MESSAGE.c:756
 af6:	4b23      	ldr	r3, [pc, #140]	(b84 <Show+0xb84>)
 af8:	240a      	movs	r4, #10
 afa:	f883 4075 	strb.w	r4, [r3, #117]
C:\Documents and Settings\jarek\Pulpit\Privet\Magisterka\Programy\1\um0427\FWLib\project/MESSAGE.c:757
 afe:	2009      	movs	r0, #9
 b00:	4621      	mov	r1, r4
 b02:	4a22      	ldr	r2, [pc, #136]	(b8c <Show+0xb8c>)
 b04:	2300      	movs	r3, #0
 b06:	f7ff fffe 	bl	0 <Show>
C:\Documents and Settings\jarek\Pulpit\Privet\Magisterka\Programy\1\um0427\FWLib\project/MESSAGE.c:758
 b0a:	2017      	movs	r0, #23
 b0c:	4621      	mov	r1, r4
 b0e:	4a20      	ldr	r2, [pc, #128]	(b90 <Show+0xb90>)
 b10:	2300      	movs	r3, #0
 b12:	f7ff fffe 	bl	0 <Show>
C:\Documents and Settings\jarek\Pulpit\Privet\Magisterka\Programy\1\um0427\FWLib\project/MESSAGE.c:759
 b16:	2004      	movs	r0, #4
 b18:	e7c6      	b.n	aa8 <Show+0xaa8>
C:\Documents and Settings\jarek\Pulpit\Privet\Magisterka\Programy\1\um0427\FWLib\project/MESSAGE.c:762
 b1a:	4b1a      	ldr	r3, [pc, #104]	(b84 <Show+0xb84>)
 b1c:	2009      	movs	r0, #9
 b1e:	f883 0075 	strb.w	r0, [r3, #117]
C:\Documents and Settings\jarek\Pulpit\Privet\Magisterka\Programy\1\um0427\FWLib\project/MESSAGE.c:763
 b22:	210a      	movs	r1, #10
 b24:	4a19      	ldr	r2, [pc, #100]	(b8c <Show+0xb8c>)
 b26:	2300      	movs	r3, #0
 b28:	f7ff fffe 	bl	0 <Show>
C:\Documents and Settings\jarek\Pulpit\Privet\Magisterka\Programy\1\um0427\FWLib\project/MESSAGE.c:764
 b2c:	2017      	movs	r0, #23
 b2e:	210a      	movs	r1, #10
 b30:	4a17      	ldr	r2, [pc, #92]	(b90 <Show+0xb90>)
 b32:	2300      	movs	r3, #0
 b34:	f7ff fffe 	bl	0 <Show>
C:\Documents and Settings\jarek\Pulpit\Privet\Magisterka\Programy\1\um0427\FWLib\project/MESSAGE.c:765
 b38:	2003      	movs	r0, #3
 b3a:	e7b5      	b.n	aa8 <Show+0xaa8>
C:\Documents and Settings\jarek\Pulpit\Privet\Magisterka\Programy\1\um0427\FWLib\project/MESSAGE.c:768
 b3c:	4b11      	ldr	r3, [pc, #68]	(b84 <Show+0xb84>)
 b3e:	2208      	movs	r2, #8
 b40:	f883 2075 	strb.w	r2, [r3, #117]
C:\Documents and Settings\jarek\Pulpit\Privet\Magisterka\Programy\1\um0427\FWLib\project/MESSAGE.c:769
 b44:	2009      	movs	r0, #9
 b46:	210a      	movs	r1, #10
 b48:	4a10      	ldr	r2, [pc, #64]	(b8c <Show+0xb8c>)
 b4a:	2300      	movs	r3, #0
 b4c:	f7ff fffe 	bl	0 <Show>
C:\Documents and Settings\jarek\Pulpit\Privet\Magisterka\Programy\1\um0427\FWLib\project/MESSAGE.c:770
 b50:	2017      	movs	r0, #23
 b52:	210a      	movs	r1, #10
 b54:	4a0e      	ldr	r2, [pc, #56]	(b90 <Show+0xb90>)
 b56:	2300      	movs	r3, #0
 b58:	f7ff fffe 	bl	0 <Show>
C:\Documents and Settings\jarek\Pulpit\Privet\Magisterka\Programy\1\um0427\FWLib\project/MESSAGE.c:771
 b5c:	2002      	movs	r0, #2
 b5e:	e7a3      	b.n	aa8 <Show+0xaa8>
C:\Documents and Settings\jarek\Pulpit\Privet\Magisterka\Programy\1\um0427\FWLib\project/MESSAGE.c:774
 b60:	4b08      	ldr	r3, [pc, #32]	(b84 <Show+0xb84>)
 b62:	2207      	movs	r2, #7
 b64:	f883 2075 	strb.w	r2, [r3, #117]
C:\Documents and Settings\jarek\Pulpit\Privet\Magisterka\Programy\1\um0427\FWLib\project/MESSAGE.c:775
 b68:	2009      	movs	r0, #9
 b6a:	210a      	movs	r1, #10
 b6c:	4a07      	ldr	r2, [pc, #28]	(b8c <Show+0xb8c>)
 b6e:	2300      	movs	r3, #0
 b70:	f7ff fffe 	bl	0 <Show>
C:\Documents and Settings\jarek\Pulpit\Privet\Magisterka\Programy\1\um0427\FWLib\project/MESSAGE.c:776
 b74:	2017      	movs	r0, #23
 b76:	210a      	movs	r1, #10
 b78:	4a05      	ldr	r2, [pc, #20]	(b90 <Show+0xb90>)
 b7a:	2300      	movs	r3, #0
 b7c:	f7ff fffe 	bl	0 <Show>
C:\Documents and Settings\jarek\Pulpit\Privet\Magisterka\Programy\1\um0427\FWLib\project/MESSAGE.c:777
 b80:	2001      	movs	r0, #1
 b82:	e791      	b.n	aa8 <Show+0xaa8>
	...
 b8c:	00000052 	.word	0x00000052
 b90:	0000005b 	.word	0x0000005b
C:\Documents and Settings\jarek\Pulpit\Privet\Magisterka\Programy\1\um0427\FWLib\project/MESSAGE.c:780
 b94:	4b14      	ldr	r3, [pc, #80]	(be8 <Show+0xbe8>)
 b96:	2202      	movs	r2, #2
 b98:	f883 2075 	strb.w	r2, [r3, #117]
C:\Documents and Settings\jarek\Pulpit\Privet\Magisterka\Programy\1\um0427\FWLib\project/MESSAGE.c:781
 b9c:	2000      	movs	r0, #0
 b9e:	f7ff fffe 	bl	0 <Show>
C:\Documents and Settings\jarek\Pulpit\Privet\Magisterka\Programy\1\um0427\FWLib\project/MESSAGE.c:782
 ba2:	2017      	movs	r0, #23
 ba4:	210a      	movs	r1, #10
 ba6:	4a11      	ldr	r2, [pc, #68]	(bec <Show+0xbec>)
 ba8:	2300      	movs	r3, #0
 baa:	f7ff fffe 	bl	0 <Show>
C:\Documents and Settings\jarek\Pulpit\Privet\Magisterka\Programy\1\um0427\FWLib\project/MESSAGE.c:783
 bae:	2009      	movs	r0, #9
 bb0:	210a      	movs	r1, #10
 bb2:	4a0f      	ldr	r2, [pc, #60]	(bf0 <Show+0xbf0>)
 bb4:	e741      	b.n	a3a <Show+0xa3a>
C:\Documents and Settings\jarek\Pulpit\Privet\Magisterka\Programy\1\um0427\FWLib\project/MESSAGE.c:790
 bb6:	490c      	ldr	r1, [pc, #48]	(be8 <Show+0xbe8>)
 bb8:	f891 3075 	ldrb.w	r3, [r1, #117]
 bbc:	2b02      	cmp	r3, #2
 bbe:	d002      	beq.n	bc6 <Show+0xbc6>
 bc0:	2b03      	cmp	r3, #3
 bc2:	d007      	beq.n	bd4 <Show+0xbd4>
 bc4:	e00b      	b.n	bde <Show+0xbde>
C:\Documents and Settings\jarek\Pulpit\Privet\Magisterka\Programy\1\um0427\FWLib\project/MESSAGE.c:792
 bc6:	698a      	ldr	r2, [r1, #24]
 bc8:	6a0b      	ldr	r3, [r1, #32]
 bca:	6013      	str	r3, [r2, #0]
C:\Documents and Settings\jarek\Pulpit\Privet\Magisterka\Programy\1\um0427\FWLib\project/MESSAGE.c:793
 bcc:	6b0b      	ldr	r3, [r1, #48]
 bce:	4798      	blx	r3
C:\Documents and Settings\jarek\Pulpit\Privet\Magisterka\Programy\1\um0427\FWLib\project/MESSAGE.c:794
 bd0:	2200      	movs	r2, #0
 bd2:	e005      	b.n	be0 <Show+0xbe0>
C:\Documents and Settings\jarek\Pulpit\Privet\Magisterka\Programy\1\um0427\FWLib\project/MESSAGE.c:797
 bd4:	698a      	ldr	r2, [r1, #24]
 bd6:	69cb      	ldr	r3, [r1, #28]
 bd8:	6013      	str	r3, [r2, #0]
C:\Documents and Settings\jarek\Pulpit\Privet\Magisterka\Programy\1\um0427\FWLib\project/MESSAGE.c:798
 bda:	6b4b      	ldr	r3, [r1, #52]
 bdc:	e7f7      	b.n	bce <Show+0xbce>
C:\Documents and Settings\jarek\Pulpit\Privet\Magisterka\Programy\1\um0427\FWLib\project/MESSAGE.c:802
 bde:	2211      	movs	r2, #17
 be0:	4b04      	ldr	r3, [pc, #16]	(bf4 <Show+0xbf4>)
 be2:	701a      	strb	r2, [r3, #0]
C:\Documents and Settings\jarek\Pulpit\Privet\Magisterka\Programy\1\um0427\FWLib\project/MESSAGE.c:808
 be4:	e8bd 817e 	ldmia.w	sp!, {r1, r2, r3, r4, r5, r6, r8, pc}
 be8:	00000000 	.word	0x00000000
 bec:	0000005b 	.word	0x0000005b
 bf0:	00000052 	.word	0x00000052
 bf4:	00000000 	.word	0x00000000
